:100000000C9485090C94BA090C94BA090C94BA0999
:100010000C94BA090C94BA090C94BA090C94BA0954
:100020000C94BA090C94BA090C94BA090C94A31A4A
:100030000C94BA090C94BA090C94BA090C94CD1614
:100040000C94BA090C94BA090C94BA090C94BA0924
:100050000C947A430C949D430C94BA090C94BA09FD
:100060000C94BA090C94BA090C94BA090C94BA0904
:100070000C94BA090C94BA090C94BA090C94BA09F4
:100080000C94BA090C94BA090C94BA09436C6561D2
:1000900072696E67205374617473000A696E7661C9
:1000A0006C696420646174650A005265706F7274D3
:1000B00020696E74657276616C3D25640A20456E18
:1000C000746572206E65773A20000A53657474690E
:1000D0006E67204D5050542062617420676F616CD0
:1000E0002025730A000A53657474696E67204D50A9
:1000F0005054204D6F64652025730A000A536574BF
:1001000074696E6720457870657274204D6F646500
:100110002025730A0025642D253032643A253032BB
:10012000643A25303264004C6F61642020252D38FC
:100130002E316620202020252D382E316620252DB9
:10014000382E316620202020252D382E316600499A
:100150006E20202020252D382E31662020202025BD
:100160002D382E316620252D382E31662020202076
:10017000252D382E31660020202020202043686164
:1001800072676528416829202050777228572920F6
:1001900020205065616B5077722857292020456ECA
:1001A0006572677928576829206F76657220252E39
:1001B00030662073656300252D362E326620252D8E
:1001C000342E32660A00252D362E326620252D3635
:1001D0002E326620252D362E326620252D362E32E3
:1001E00066252D362E326620252D342E32662025AA
:1001F0002D352E3166202564202564202564202598
:100200002D362E326620252D342E32660A000A53F2
:10021000657474696E67204C43442025730A006D31
:100220007070745F7363616E5F696E74657276611E
:100230006C3D2564206D696E0A20456E74657220E0
:100240006E65773A20004F4B0A000A536574746953
:100250006E672041545820534220506F77657220BA
:1002600025730A000A53657474696E6720415458F7
:1002700020506F7765722025730A0041545820532F
:1002800069672E205057525F4F4B2025730A00415B
:100290005458205369672E2050535F4F4E2020251D
:1002A000730A004154582050575220202020202506
:1002B000730A0041545820534220505752202025A1
:1002C000730A004368616E6765204F7363696C6CE5
:1002D00061746F722E204E6F77204F534343414C11
:1002E0003D25640A20456E746572206E65773A205C
:1002F0000020554252524C3D25642000204F53436C
:1003000043414C3D2564200020556E757365642083
:10031000737461636B203D25640020467573653AF4
:100320002065653D253032782068663D253032787D
:10033000206C663D25303278206C623D2530327865
:10034000004D43553D2530366C7800252D31306CFD
:100350007520252D31306C7520252D31306C7520A0
:10036000252D31306C7520252D31306C7520252DD3
:1003700031306C7520252D31306C750A00565F695F
:100380006E3E4D617820202056206261743E4D61A2
:100390007820204120696E3E4D6178202020412048
:1003A0006C6F61643E4D61782054206261743E4DF3
:1003B0006178202054206D69737320636E74204C23
:1003C000564420636E740A00446174652020202026
:1003D00020202054696D6520202020204261742057
:1003E000202020476F616C202020496E2020202093
:1003F00020615F696E202050574D20207077725F1A
:10040000696E20206D70707420207077722D646981
:1004100066660A0044617465202020202020205454
:10042000696D652020202020416828696E292020E0
:10043000204168286C6F61642920205028696E294A
:10044000202050286C6F61642920205128696E2972
:10045000202051286C6F6164290A00446174652072
:1004600020202020202054696D652020202020425B
:10047000617420202020476F616C202020496E206D
:1004800020202020615F696E202050574D2020548D
:100490005F426174207431202074322020765F6CBA
:1004A0006F616420615F6C6F61640A0043757272F2
:1004B000656E742064656275673D3078255820202C
:1004C0004E65773A2000445F504F5745523D307893
:1004D00025780A00445F4C45443D307825780A0071
:1004E000445F4F573D307825780A00445F4D5050A7
:1004F000545F5343414E5F424553543D3078257815
:100500000A00445F4D5050545F5343414E3D307894
:1005100025780A00445F4D5050543D307825780AC4
:1005200000445F4C4F41443D307825780A00445FD9
:100530004348415247453D307825780A00445F4F93
:100540005045523D307825780A00456E746572201A
:100550004F6E2D426F6172642074656D70207365FB
:100560006E736F72206964783A2000456E7465720C
:1005700020426174746572792074656D70207365B2
:100580006E736F72206964783A20004261747465FA
:1005900072792054656D70203D2025352E3266001D
:1005A000765F6C76645F687973743D25352E3266AC
:1005B0000A20456E746572206E65773A2000765F7A
:1005C0006C76643D25352E32660A20456E74657260
:1005D000206E65773A20004C6F61642063757272FB
:1005E000656E74206C696D69743D25352E32660A1E
:1005F00020456E746572206E65773A2000496E70F2
:1006000075742063757272656E74206C696D69749F
:100610003D25352E32660A20456E746572206E6562
:10062000773A2000765F676F616C5F6C6F61643D45
:1006300025352E32660A20456E746572206E657708
:100640003A2000765F676F616C3D25352E32660A71
:1006500020456E746572206E65773A2000666C7472
:100660005F666163746F723D25352E32660A2045E0
:100670006E746572206E65773A2000666C74206631
:100680006163746F7220636F6E74726F6C73207429
:10069000686520706572696F64206265666F726557
:1006A000206E65787420626F6F7374207065726954
:1006B0006F640A00506C65617365207365742079FE
:1006C0006F757220666978656420766F6C746167F7
:1006D0006525730A000A53657474696E672046695C
:1006E00078656420566F6C74616765204D6F646532
:1006F0002025730A006174787320202D207365749F
:100700002041545820534220706F77657220257322
:100710000A006174787020202D2041545820706F99
:100720007765722025730A00726920202D2072657A
:10073000706F727420696E74657276616C20696E78
:10074000207365630A0D00727320202D207265737B
:10075000746F72652064656661756C74207365746E
:1007600074696E67730A0D006F7720202D206F77F4
:100770002D6275732064756D700A0D006D692020FF
:100780002D20736574204D505054207363616E208A
:10079000696E74657276616C0A006D6220202D208E
:1007A000736574204D505054206261747465727981
:1007B0002025730A006D7420202D20736574204D50
:1007C0005050542025730A006C7020202D20736532
:1007D00074204C43442025730A00646920202D2096
:1007E000646973636F6E6E65637420696E7075748F
:1007F000206D616E75616C6C790A0D006369202053
:100800002D20636F6E6E65637420696E7075742041
:100810006D616E75616C6C790A0D00646C20202D21
:1008200020646973636F6E6E656374206C6F6164BE
:10083000206D616E75616C6C790A0D00636C20200F
:100840002D20636F6E6E656374206C6F6164206D24
:10085000616E75616C6C790A0D00762020202D2068
:1008600076657273696F6E0A0D00752020202D2049
:10087000757074696D650A0D00747320202D2074E5
:10088000696D65207365740A0D00636320202D2057
:1008900063686172676520737461747320636C654B
:1008A00061720A0D00637320202D206368617267F6
:1008B000652073746174730A0D00742020202D204C
:1008C00074696D652073686F770A0D006465202078
:1008D0002D2064656275670A0D00737320202D203A
:1008E0007374617475732073756D6D6172790A0D1F
:1008F00000626D20202D206261747465727920730E
:1009000075626D656E750A0D00682020202D2068C7
:10091000656C700A0D00756E6B6E6F776E20636D7F
:10092000640A006D2020202D206261636B20746FAB
:10093000206D61696E206D656E750A0D007268200C
:10094000202D207265636F6E6E6563742068797305
:100950007465726573697320766F6C746167650A7C
:100960000D00647620202D20646973636F6E6E65C0
:10097000637420766F6C746167650A0D00766C2075
:10098000202D20766F6C74616765206C6F61642028
:10099000676F616C0A0D00666620202D20666C6F03
:1009A000617420706572696F6420666163746F7230
:1009B0000A0D00766720202D20766F6C74616765C4
:1009C00020676F616C0A0D00667620202D20626121
:1009D000747465727920666978656420766F6C74CA
:1009E000616765206D6F64650A0D00626120202DCE
:1009F000206261747465727920766F6C74616765CA
:100A000020706172616D730A0D00746920202D20C1
:100A1000626174746572792073656E736F72206F92
:100A20006E652D7769726520696E6465780A0D00C0
:100A3000746520202D20626174746572792074655C
:100A40006D70657261747572650A0D0063612020B6
:100A50002D2063616C69627261746520766F6C74BD
:100A60006167652072656164696E67730A0D006174
:100A70006C20202D206C696D6974206C6F6164207E
:100A800063757272656E740A0D00616920202D20F5
:100A90006C696D697420696E70757420637572720B
:100AA000656E740A0D00646520202D2064656275F2
:100AB000670A0D00682020202D2068656C700A0DE3
:100AC00000426F6F737420566F6C746167652061AC
:100AD0007420323043203D25352E32660A20456E83
:100AE000746572204E65773A2000466C6F61742001
:100AF000566F6C7461676520617420323043203D0D
:100B000025352E32660A20456E746572204E657753
:100B10003A2000496E2043757272656E743D25352A
:100B20002E32660A20456E74657220636F7272659C
:100B3000637465643A20004C6F616420437572727F
:100B4000656E743D25352E32660A20456E746572D9
:100B500020636F727265637465643A20004C6F6144
:100B60006420566F6C746167653D25352E32660AC8
:100B700020456E74657220636F727265637465647C
:100B80003A2000496E70757420566F6C7461676509
:100B90003D25352E32660A20456E74657220636FDE
:100BA000727265637465643A2000426174746572A0
:100BB0007920566F6C746167653D25352E32660A63
:100BC00020456E74657220636F727265637465642C
:100BD0003A20005265706F727420696E7465727687
:100BE000616C203D25356420730A004C6F616420E0
:100BF000617665726167652063757272656E7420D7
:100C00003D25352E336620410A004C6F6164207605
:100C10006F6C7461676520676F616C203D25352EB0
:100C20003166560A004D505054207363616E20693E
:100C30006E74657276616C203D2564206D696E0A64
:100C4000004D505054207363616E3A2050574D2030
:100C500075736564203D2025642C206265737420C3
:100C60003D25642C205057523D25352E33660A0011
:100C70004D50505420765F626174203D25640A0017
:100C80004D505054206C6F636B2F6E6F6C6F636BA5
:100C9000203D256C752F256C750A0054656D7020FC
:100CA00062617474657279203D25362E3266204368
:100CB000202844656661756C74290A0054656D705E
:100CC0002073656E736F72206572726F72203D259E
:100CD0006420430A00202844656661756C742920ED
:100CE0005741524E494E472074656D702073656EB2
:100CF000736F72206964206E6F7420636F6E666913
:100D000067757265640054656D7020626174746506
:100D10007279203D25362E3266204300566F6C7462
:100D2000616765206C6F6164207265636F6E6E65CC
:100D30006374206F6666736574203D25352E3266B8
:100D400020560A00496E707574206973206D616EBB
:100D500075616C6C7920646973636F6E6E65637422
:100D600065640A004C6F6164206C6173742064696F
:100D700073636F6E6E656374656420004C6F6164AD
:100D8000206973206D616E75616C6C792064697384
:100D9000636F6E6E65637465640A004C6F616420F6
:100DA0006973206C6F7720766F6C7461676520645F
:100DB0006973636F6E6E65637465640A00566F6C69
:100DC00074616765206C6F616420646973636F6E22
:100DD0006E656374203D25352E316620560A004C21
:100DE0006173742063686172676520004D617820CB
:100DF0006C6F61642063757272656E74203D253579
:100E00002E316620410A004D617820696E7075743C
:100E10002063757272656E74203D25352E31662013
:100E2000410A0043757272656E74206C6F616420B4
:100E30003D25362E336620410A0043757272656E79
:100E40007420696E203D25362E336620410A0056F7
:100E50006F6C74616765206C6F6164203D25352E71
:100E6000326620560A00566F6C7461676520676FA2
:100E7000616C203D25352E3166560A00566F6C7424
:100E800061676520666C6F6174203D25352E316683
:100E9000560A00566F6C7461676520626F6F7374D9
:100EA000203D25352E3166560A00566F6C746167F9
:100EB0006520696E203D25352E326620560A005683
:100EC0006F6C7461676520626174203D25352E3238
:100ED0006620560A00566F6C746167652063617006
:100EE000203D25352E326620560A004C564420748B
:100EF000696D652000557074696D652000446174EA
:100F0000652000312E300D0A0020257320537461B6
:100F1000727420005254432025732C00436F707963
:100F20007269676874204865726A756C66205574CA
:100F30007665636B6C696E672C2055707073616C9D
:100F4000612053776564656E2C206865726A756CE4
:100F5000662E73650D0A004669726D7761726520B1
:100F60005665722E20362E3520323031332D3130F9
:100F70002D33310D0A0020252D382E316620252DE8
:100F8000382E316620252D382E316620252D382E1D
:100F9000316620252D382E306620252D382E3066DE
:100FA0000A004368617267652074696D6572206527
:100FB0007870697265642061667465722025752099
:100FC0007365630A00426F6F7374207265616368B2
:100FD000656420696E2025752073656320666C74D6
:100FE0002D706572696F642073657420746F20259D
:100FF00075207365630A00204D505054207363615F
:101000006E20646F6E653A2050574D20757365648D
:10101000203D202534642C2062657374203D2534E6
:10102000642C205057523D25352E33660A00204D42
:10103000505054207363616E3A2050574D207573A1
:101040006564203D202534642C207363616E203D4F
:101050002534642C205057523D25352E33660A0026
:1010600020252D362E326620252D362E326620255F
:101070002D362E326620252D342E326620253464FE
:101080002020252D372E33662025642020252D375E
:101090002E3366200A0020252D362E326620252D7F
:1010A000362E326620252D342E3266202534640AF1
:1010B0000020252D362E326620252D362E32662034
:1010C000252D362E326620252D342E3266202534ED
:1010D0006420252D352E31662025642025642025A9
:1010E0006420252D362E326620252D342E32660AB8
:1010F00000263A00253034642D253032642D253009
:10110000326420253032643A253032643A25303258
:101110006400745F626174203D2025362E32660AB9
:10112000005761726E696E672E2042617474657239
:10113000792073656E736F72206964206E6F7420FE
:101140007365740A005761726E696E672E204E6F68
:101150002074656D702073656E736F72730A005230
:101160006573657474696E6700526573746F726538
:1011700020616C6C2073657474696E67733F2079AD
:101180002F6E3A2000253034642D253032642D2511
:1011900030326420253032643A253032643A2530CA
:1011A00032640020257300204F6E2D426F617264FF
:1011B000002042617474657279002025362E3266F3
:1011C00020002530327800256420000A006E616E10
:1011D00000696E660000407A10F35A00A0724E1843
:1011E000090010A5D4E80000E87648170000E40BD9
:1011F00054020000CA9A3B000000E1F5050000809F
:10120000969800000040420F000000A086010000F8
:1012100000102700000000E8030000000064000048
:101220000000000A00000000000100000000002C87
:1012300076D888DC674F0823DFC1DFAE59E1B1B74C
:1012400096E5E3E453C63AE651997696E8E6C28419
:1012500026EB898C9B62ED407C6FFCEFBC9C9F4031
:10126000F2BAA56FA5F490055A2AF75C936B6CF956
:10127000676DC11BFCE0E40D47FEF520E6B500D02C
:10128000ED902E0300943577050080841E08000041
:10129000204E0A000000C80C333333330F986E120F
:1012A000831141EF8D2114893BE65516CFFEE6DB15
:1012B00018D1844B381BF77C1D901DA4BBE424205F
:1012C0003284725E228100C9F124ECA1E53D2749F8
:1012D0004E46494E4954594E414ECDCCCC3D0AD78D
:1012E000233C17B7D13877CC2B329595E6241FB124
:1012F0004F0A000020410000C84200401C4620BCAC
:10130000BE4CCA1B0E5AAEC59D74EDEBF3E085ECE6
:1013100090E401C08193EF3FF907E0F3D9F3112482
:101320001FBECFEFD0E4DEBFCDBF84B78093BC0338
:1013300014BE88E10FB6F8948093600010926000AC
:101340000FBE11E0A0E0B1E0EAE0F6EA00E00BBF7A
:1013500002C007900D92A23CB107D9F713E0A2ECAE
:10136000B1E001C01D92AC3BB107E1F70E94DD384E
:101370000C9403530C940000209170002C7F209358
:1013800070000097C1F081E08093A6018091B600C3
:1013900080628093B6001092B20082E08093B10028
:1013A0008091B60090E0877090700097C9F781E057
:1013B0008093700008951092A6011092B20080915F
:1013C000B6008F7D8093B60086E08093B100809157
:1013D000B60090E0877090700097C9F781E0809325
:1013E00070000895AF92BF92CF92DF92EF92FF927A
:1013F0000F931F93CF93DF937B018C018DB79EB723
:101400000A970FB6F8949EBF0FBE8DBFCDB7DEB75B
:10141000219685E191E0EDB7FEB792838183C80103
:10142000B70120E831E541E050E00E94BF4B3B832B
:101430002A8330E1A32E3EE0B32EC12CD12CA6018D
:1014400095010E94BF4B332727FD30953D832C83A8
:10145000C801B701A60195010E94BF4B2CE3A22E43
:10146000B12CC12CD12CA60195010E94BF4B332772
:1014700027FD30953F832E83C801B701A601950152
:101480000E94BF4B772767FD7095798768870E9418
:10149000FF4E8DB79EB708960FB6F8949EBF0FBE4D
:1014A0008DBF8BEC91E1EDB7FEB7928381830E94F3
:1014B000FF4E0F900F90DF91CF911F910F91FF90F2
:1014C000EF90DF90CF90BF90AF900895EDEBF3E0F9
:1014D00080E4EF3FF80709F0A8F420E030E005C011
:1014E00080E4EF3FF80709F058F431968081853C9D
:1014F000B9F72F5F3F4F80E4EF3FF807B1F3A8F350
:10150000C901089520E030E0FBCF009749F4109224
:1015100046011092C2010A9A1298089A10980895EA
:1015200081E0809346010898109A0895009739F455
:101530000A9A12981092C201229A2A980895229823
:101540002A9A08956F927F928F929F92AF92BF9244
:10155000CF92DF92EF92FF920F931F93DF93CF937F
:10156000CDB7DEB729970FB6F894DEBF0FBECDBF5B
:101570001092D7018FEF89837FE3C72E72E0D72EB9
:10158000EE24FF24882462E0A62EB12CAC0EBD1EF2
:101590003E010894611C711C8E01065F1F4F9E2C3A
:1015A000C301B5010E948B4189818F3F09F485C039
:1015B0008E3F09F482C0C5010E94A641F6018087D2
:1015C000F501D701AA0FBB1FAA0FBB1FAA0FBB1F94
:1015D000AE0DBF1DA15CBD4F81918D93E017F1074A
:1015E000D9F79091BB02F60180819817D1F19394BD
:1015F0008981882369F00894E11CF11C89E090E05E
:10160000C80ED91E98E0E916F10449F648E0942E78
:10161000882089F48FEF8093BB028093BC02809373
:10162000BD028093BE028093BF028093C00280936C
:10163000C1028093C202892D29960FB6F894DEBFAD
:101640000FBECDBFCF91DF911F910F91FF90EF9013
:10165000DF90CF90BF90AF909F908F907F906F90D2
:1016600008959091BC028181981709F69091BD026E
:101670008281981709F0BBCF9091BE0283819817A1
:1016800009F0B5CF9091BF028481981709F0AFCFD0
:101690009091C0028581981709F0A9CF9091C1025D
:1016A0008681981709F0A3CF9091C202878198177D
:1016B00009F09DCF882483949ACF8093D701A8CF37
:1016C0000E94A20A8093D601089500D08BEC91E18C
:1016D000EDB7FEB7928381830E94FF4E0F900F906B
:1016E00008952F923F924F925F926F927F928F92C6
:1016F0009F92AF92BF92CF92DF92EF92FF920F93A1
:101700001F93CF93DF930E94600B8091D6018823B3
:1017100009F4BEC0CFE3D2E0AA24BB24B7EC4B2E21
:10172000B1E15B2EA2ECCA2EA1E1DA2EFAEB2F2E4C
:10173000F1E13F2E00D000D0ADB7BEB712965C925B
:101740004E9211971496BC92AE9213970E94FF4E40
:101750000F900F900F900F908501000F111F000F39
:10176000111F000F111F0A0D1B1D015C1D4FC80129
:101770000E94EB42FC01BF01882777FD8095982FDE
:101780000E94754A3B014C01780100E010E0D7014E
:101790008D917D0100D000D0EDB7FEB73196ADB789
:1017A000BEB71296DC92CE921197828313820E946A
:1017B000FF4E0F5F1F4F0F900F900F900F9008304C
:1017C000110529F700D000D000D00DB71EB70F5F6C
:1017D0001F4FEDB7FEB732822182662D772D882DFF
:1017E000992D20E030E048EC52E40E94DA49D8011B
:1017F00012966D937D938D939C9315970E94FF4E47
:10180000888129813A81EB817C816D815E814F8164
:10181000ADB7BEB716960FB6F894BEBF0FBEADBF3C
:101820009091BB02981709F47AC09091170398170A
:1018300009F444C088858823F1F180E091E000D06C
:1018400000D0E3EAF1E1ADB7BEB71296FC93EE9398
:10185000119714969C938E9313970E94FF4E0F90AE
:101860000F90EBECF1E1ADB7BEB71296FC93EE939F
:1018700011970E94FF4E0894A11CB11C29968091DB
:10188000D60190E00F900F90A816B9060CF452CF35
:10189000DF91CF911F910F91FF90EF90DF90CF904C
:1018A000BF90AF909F908F907F906F905F904F9080
:1018B0003F902F90089589E091E0C1CF8091180367
:1018C000821709F0B7CF80911903831709F0B2CFBF
:1018D00080911A038E1709F0ADCF80911B038717F3
:1018E00009F0A8CF80911C03861709F0A3CF80913F
:1018F0001D03851709F09ECF80911E03841709F000
:1019000099CF00D0E7EAF1E1ADB7BEB71296FC93EC
:10191000EE9311970E94FF4E0F900F908BCF9091F6
:10192000BC02921709F081CF9091BD02931709F084
:101930007CCF9091BE029E1709F077CF9091BF02A5
:10194000971709F072CF9091C002961709F06DCFEA
:101950009091C102951709F068CF9091C202941737
:1019600009F063CF00D021EB31E1EDB7FEB7328350
:1019700021830E94FF4E888129813A81EB817C81FD
:101980006D815E814F810F900F904FCFEAE7F0E0BD
:1019900080E8808380818760808310927B0088EF5D
:1019A00080937E00808188608083808180648083D2
:1019B000089580937C0080917C00806C80937C00F3
:1019C00086E080937A0080917A00806880937A0024
:1019D00080917A00806480937A0080917A0086FDFD
:1019E000FCCF88E090E060E070E020917A00206415
:1019F00020937A0020917A0026FDFCCF2091780078
:101A000030917900620F731F019779F780917A0006
:101A10008F7780937A00769567957695679576951A
:101A2000679580E090E00E94734A0895CF92DF921C
:101A3000EF92FF920F931F93CF93DF937B018C0163
:101A40006A01E901FA018081882371F4C801B701B4
:101A500020E030E0A9010E94254B18160CF054C07C
:101A60006497109201020CC0C801B70120E030E079
:101A7000A9010E94254B181604F5649610920102E4
:101A80008091EC019091ED01A091EE01B091EF01F8
:101A90000196A11DB11D8093EC019093ED01A093DF
:101AA000EE01B093EF01CE01DF91CF911F910F9125
:101AB000FF90EF90DF90CF900895C801B70120E02C
:101AC00030E0A9010E94D64987FD31C08091010212
:101AD0008F5F80930102823098F2815080930102DF
:101AE0008091E8019091E901A091EA01B091EB01A8
:101AF0000196A11DB11D8093E8019093E901A09387
:101B0000EA01B093EB01CFCFC801B70120E030E08C
:101B1000A9010E94D64987FFD9CF81E0F6018083D1
:101B20006496809101028F5F80930102D4CF649705
:101B3000F6011082809101028F5F80930102CBCF6A
:101B4000EF92FF920F931F93CF93DF936091130354
:101B50007091140380911503909116032091FF0258
:101B60003091000340910103509102030E94254BE4
:101B700018160CF580919A0190919B0123E08F3FFC
:101B8000920728F580919A0190919B01E0919C0128
:101B9000F0919D0190939901809398018091980113
:101BA0009091990191838083DF91CF911F910F9143
:101BB000FF90EF9008958091DE01882359F0809185
:101BC0009A0190919B0133E08F3F9307D8F28FEFFA
:101BD00093E0DCCF60910F037091100380911103AB
:101BE00090911203E0907101F090720100917301E5
:101BF00010917401A80197010E94254B18160CF052
:101C000063C060910F037091100380911103909154
:101C10001203A80197010E94714920E030E0A90158
:101C20000E94254B18160CF057C060910F0370915D
:101C300010038091110390911203A80197010E9453
:101C4000714920E030E048E452E40E94294B0E94B0
:101C5000474A8091980190919901860F971F97FDAF
:101C6000F6C020919A0130919B012817390720F482
:101C700080919A0190919B01E0919C01F0919D01CE
:101C80009093990180939801809198019091990186
:101C9000918380838091A3029091A402A091A502D8
:101CA000B091A6020196A11DB11D8093A30290934D
:101CB000A402A093A502B093A602DF91CF911F9139
:101CC0000F91FF90EF900895809100021816D4F4C0
:101CD00081508093000268CF60910F0370911003D0
:101CE0008091110390911203A80197010E947149FC
:101CF000905820E030E048E452E40E94294B0E94D2
:101D0000474AA7CF8091FE019091FF0101969093E1
:101D1000FF018093FE0180918F0290919002A0912B
:101D20009102B091920280930B0390930C03A093C5
:101D30000D03B0930E0380918B01882309F4A6C094
:101D40006091130370911403809115039091160311
:101D500020910F0330911003409111035091120311
:101D60000E94294B9B01AC0120938F02309390027B
:101D700040939102509392026091610170916201CF
:101D800080916301909164012091130330911403B9
:101D900040911503509116030E94714920E030E0F4
:101DA000A9010E94254B18160CF054C060916101E6
:101DB00070916201809163019091640120911303FD
:101DC0003091140340911503509116030E947149FC
:101DD00020E030E048E452E40E94294B0E94474A48
:101DE000E62EE7017E01F72EE701CF31D10510F095
:101DF000CEE1D0E06091FF02709100038091010379
:101E000090910203E0901303F090140300911503E6
:101E1000109116032DEC3CEC4CE45EE30E947149FA
:101E2000A80197010E94254B1816CCF180919801CA
:101E3000909199018C0F9D1F97FDFFC020919A01F1
:101E400030919B012817390708F49CCE9FCE80E083
:101E500090E012CF60916101709162018091630105
:101E60009091640120911303309114034091150364
:101E7000509116030E947149905820E030E048E4E8
:101E800052E40E94294B0E94474AAACF6091FF0268
:101E900070910003809101039091020359CF6091EA
:101EA00013037091140380911503909116032091F0
:101EB00061013091620140916301509164010E947F
:101EC000254B18169CF580919801909199018C0FE3
:101ED0009D1F97FDB5C020919A0130919B01281755
:101EE000390720F480919A0190919B01E0919C0127
:101EF000F0919D01909399018093980180919801B0
:101F000090919901918380836091B7027091B8029A
:101F10008091B9029091BA0220E030E0A9010E94BC
:101F2000D64987FF41CE1092D1013ECE6091130376
:101F30007091140380911503909116032091610113
:101F40003091620140916301509164010E94D64931
:101F500087FF2ACE80918A01882309F466C0809188
:101F6000D101882309F4DFC060918F027091900243
:101F700080919102909192022091B7023091B80223
:101F80004091B9025091BA020E94254B18160CF4E8
:101F9000B1C02091FC013091FD012115310509F0FE
:101FA00052C0809198019091990190933E02809344
:101FB0003D0284E690E03093C7022093C6029093DE
:101FC000FD018093FC0120919A0130919B0128171B
:101FD000390720F480919A0190919B01E0919C0136
:101FE000F0919D01909399018093980180919801BF
:101FF000909199019183808380918F0290919002BA
:10200000A0919102B09192028093210390932203B8
:10201000A0932303B09324038091200388608093CE
:10202000200387E080930002BFCD809198019091BA
:1020300099018C1B9D0B97FF01CF80E090E0A6CD0E
:1020400080E090E053CFC9018C599F4F43E08F3F10
:10205000940708F4B0CF1092D1018091C4029091FE
:10206000C50297FDB7C020919A0130919B012817B6
:10207000390720F480919A0190919B01E0919C0195
:10208000F0919D019093990180939801809198011E
:1020900090919901918380838091B7029091B802C9
:1020A000A091B902B091BA028093210390932203C8
:1020B000A0932303B093240380E090E0A0E8BFEB5B
:1020C0008093B7029093B802A093B902B093BA027A
:1020D0008091C4029091C5029093C7028093C6027A
:1020E0001092FD011092FC01809120038061809389
:1020F000200397CF2091FC013091FD013093C50260
:102100002093C40280918F0290919002A09191023D
:10211000B09192028093B7029093B802A093B90253
:10212000B093BA023ACF85E08093000260918F02AB
:1021300070919002809191029091920220910B03F4
:1021400030910C0340910D0350910E03C091980102
:10215000D09199010E9471494BEA51E09E010E9481
:10216000160D909399018093980180919801909118
:10217000990123E08F3F920734F16091130370912E
:1021800014038091150390911603E0906101F09083
:10219000620100916301109164012DEC3CEC4CE470
:1021A0005EE30E947249A80197010E94D64987FF09
:1021B00014C08091C4029091C502909399018093BC
:1021C00098011092AB01809198019091990197FD2F
:1021D00034CF34CE80E090E051CF8FEF93E09093F6
:1021E000990180939801EFCFCF92DF92EF92FF9207
:1021F0000F931F93CF93DF9360919302709194029A
:10220000809195029091960220917501309176010E
:1022100040917701509178010E94254B1816ECF5FA
:1022200080918C0190918D0184539F4F97FDBDC08B
:1022300020918E0130918F012817390720F4809169
:102240008E0190918F01E0919001F0919101909316
:102250008D0180938C0180918C0190918D019183EF
:1022600080838091A7029091A802A091A902B091C9
:10227000AA020196A11DB11D8093A7029093A80206
:10228000A093A902B093AA02DF91CF911F910F9161
:10229000FF90EF90DF90CF9008958091DD0188232B
:1022A000E1F080918E0190918F0123E08F3F9207A2
:1022B00008F07EC080918E0190918F01E091900195
:1022C000F091910190938D0180938C0180918C010C
:1022D00090918D0191838083D7CF8091DC018823F9
:1022E00001F7E0906501F09066010091670110919F
:1022F00068012091310230913202409133025091B5
:102300003402C801B7010E94714920E030E0A90100
:102310000E94254B18160CF068C0209131023091B4
:1023200032024091330250913402C801B7010E9439
:10233000714920E030E048E452E40E94294B0E94B9
:10234000474AC62EE6016E01D72EE601C430D105FC
:1023500010F0C3E0D0E02091310230913202409180
:10236000330250913402C801B7010E94D64987FF59
:1023700022C080918C0190918D018C0F9D1F33E0C4
:102380008D3F930708F047C080918C0190918D019B
:102390008C0F9D1F97FD26C020918E0130918F01DB
:1023A0002817390708F486CF89CF80E090E04BCF1B
:1023B0008FEF93E083CF2091310230913202409130
:1023C000330250913402C801B7010E94254B181600
:1023D0000CF05ACF80918C0190918D018C1B9D0B3C
:1023E00097FFDACF80E090E069CF20913102309101
:1023F00032024091330250913402C801B7010E9469
:102400007149905820E030E048E452E40E94294BA2
:102410000E94474A96CF80918C0190918D01CCEF1C
:10242000D3E0C81BD90BB0CF94B1936094B995B1E8
:10243000936095B9833081F0843038F0863091F024
:10244000873039F0853041F00895813021F08230B5
:1024500028F02998089529982898089585B18360CF
:1024600085B90895299885B1817085B90895CF936C
:10247000DF938FE192E020911F0230912002FC0156
:102480003197A081FC0132977081FC013397608104
:10249000FC01349750810597EC014881EDB7FEB7F8
:1024A0003E970FB6F894FEBF0FBEEDBF319685E89C
:1024B00091E1CDB7DEB79A83898333832283A483E6
:1024C0001582768317826087118652871386448728
:1024D00015860E94FF4EEDB7FEB73E960FB6F894F4
:1024E000FEBF0FBEEDBFDF91CF910895AAE1B2E02C
:1024F000E9EAF3E087E001900D928150E1F7089559
:10250000CF93DF93ECE9F1E0A0919C01B0919D01A4
:10251000EF0122978881998134979183808380810C
:10252000918111969C938E935D98DF91CF91089540
:10253000E0E8F0E020EC20832081236020832AE083
:1025400020938100A8E8B0E011969C938E938D9122
:102550009C911197559A8081806380838FEF91E0E1
:1025600090938D0180938C0190938B0080938A00CF
:10257000549A81E080936F008FEF93E090938F01E6
:1025800080938E0190939B0180939A017894089593
:102590008FEF81B911B812B884B914B815B887B9DA
:1025A00017B818B88AB91AB81BB80F980E980D98B2
:1025B0000C980B9888EF80937E00399A419A389A4C
:1025C000409A579A5F9A8091C40181FF0BC0809115
:1025D0004701882309F4D2C081E090E00E94960A66
:1025E0008091C40180FF09C080914601882309F0D1
:1025F000CCC080E090E00E94850A81E090E00E94DB
:10260000BC0981E791E06DE270E044E050E00E9497
:10261000B44F85E791E061E370E044E050E00E9450
:10262000B44F89E791E066E370E044E050E00E9437
:10263000B44F81E691E06DE170E044E050E00E942B
:10264000B44F85E691E061E270E044E050E00E9422
:10265000B44F89ED91E065E370E041E050E00E9405
:10266000B44F8BEB92E066E470E049E050E00E94EA
:10267000B44F87E193E06FE470E049E050E00E94DE
:10268000B44F88E591E06CE070E044E050E00E94D7
:10269000B44F8CE591E060E170E044E050E00E94CE
:1026A000B44F85EC91E064E170E044E050E00E94BA
:1026B000B44F89EC91E068E170E044E050E00E94A2
:1026C000B44F80E591E064E070E044E050E00E94A7
:1026D000B44F84E591E068E070E044E050E00E948F
:1026E000B44F8CE491E060E070E044E050E00E9480
:1026F000B44F8DE791E06AE370E044E050E00E945F
:10270000B44F89E691E065E270E044E050E00E9459
:10271000B44F8DE691E069E270E044E050E00E9441
:10272000B44F82E891E06EE370E044E050E00E9434
:10273000B44F8AE891E062E470E044E050E00E9427
:10274000B44F8BE891E063E470E044E050E00E9415
:10275000B44F80E691E06CE170E041E050E00E940F
:10276000B44F85EE91E064E470E042E050E00E94F6
:10277000B44F8FEF93E00E949812089580E090E0AC
:102780000E94960A8091C4012DCF81E090E00E94C2
:10279000850A33CFEF92FF920F931F93CF93DF936E
:1027A0008091D601882309F4ADC08091BB028F3F90
:1027B00009F456C08BEB92E00E94EB429C01B901F8
:1027C000882777FD8095982F0E94754A20E030E099
:1027D00048EC52E40E94DA49E62EF72E082F192F12
:1027E0002091D2013091D30126FDB7C0C801B701B5
:1027F00020E030E048EA52E40E94254B1816FCF431
:102800001092D6018091AB029091AC02A091AD02E2
:10281000B091AE020196A11DB11D8093AB029093C1
:10282000AC02A093AD02B093AE020F2EF0E0EF2EFB
:10283000F0E0FF2EF8EC0F2FF1E41F2FF02DF894AD
:10284000E0924801F092490100934A0110934B0134
:102850007894DF91CF911F910F91FF90EF900895A1
:102860008091BC028F3F09F0A5CF8091BD028F3FC0
:1028700009F0A0CF8091BE028F3F09F09BCF8091DD
:10288000BF028F3F09F096CF8091C0028F3F09F0C1
:1028900091CF8091C1028F3F09F08CCF8091C2020D
:1028A0008F3F09F087CF8091AB029091AC02A0914D
:1028B000AD02B091AE020196A11DB11D8093AB0295
:1028C0009093AC02A093AD02B093AE028091D2017E
:1028D0009091D30186FF36C000D081E291E1EDB73F
:1028E000FEB7928381830E94FF4E0F900F900F2EB0
:1028F000F0E0EF2EF0E0FF2EF8EC0F2FF1E41F2FA9
:10290000F02D9DCF0E94600B8091D601882309F0A5
:102910004CCF8091AB029091AC02A091AD02B091EE
:10292000AE020196A11DB11D8093AB029093AC0243
:10293000A093AD02B093AE028091D2019091D301E9
:1029400086FD2AC00F2EF0E0EF2EF0E0FF2EF8EC0F
:102950000F2FF1E41F2FF02D72CF00D000D000D048
:1029600022E131E1CDB7DEB73A832983262F372F15
:10297000482F592FEDB7FEB7238334834583568301
:102980000E94FF4E2DB73EB72A5F3F4F0FB6F89417
:102990003EBF0FBE2DBF2ACF00D085E491E1CDB759
:1029A000DEB79A8389830E94FF4E0F900F900F2EFF
:1029B000F0E0EF2EF0E0FF2EF8EC0F2FF1E41F2FE8
:1029C000F02D3DCF6091DF017091E001611571053F
:1029D00051F481E090E09093E0018093DF0168E89A
:1029E00073E1CB01089588E893E10E94984B61154B
:1029F0007105B9F761E070E0CB010895CF93DF93E3
:102A0000C091DF01D091E0012097E9F0BE0180E0A4
:102A100090E00E94734A9B01AC0160918201709129
:102A2000830180918401909185010E94DA490E947E
:102A3000474A262F372F2C173D0708F49E01C9015E
:102A4000DF91CF91089581E090E09093E001809331
:102A5000DF0120E030E040E85FE3C1E0D0E0DDCF1F
:102A60002F923F924F925F926F927F928F929F929E
:102A7000AF92BF92CF92DF92EF92FF920F931F938C
:102A8000DF93CF9300D000D0CDB7DEB73B014C0130
:102A9000209148013091490140914A0150914B01E8
:102AA00060E070E080EA91E40E94714926EA3BE927
:102AB00044EC5CE30E94294B20916D0130916E0142
:102AC00040916F01509170010E947249F62E072FBC
:102AD000182FE92E862F902FA12FBE2D89839A8340
:102AE000AB83BC83209148013091490140914A0158
:102AF00050914B0160E070E080EA91E40E947149DE
:102B000026EA3BE944EC5CE30E94294B20916901F1
:102B100030916A0140916B0150916C010E947249A1
:102B20005B016C0115012601C401B3012F2D302F6B
:102B3000412F5E2D0E94254B87FD07C08091FA0131
:102B40009091FB01009709F49DC0809186019091BE
:102B50008701009709F05CC0809120038064809316
:102B600020038091DF019091E0019093E201809336
:102B7000E1018091FA019091FB018130910559F0BA
:102B80008091F6019091F70101969093F70180935F
:102B9000F60180FD63C02092610130926201409293
:102BA00063015092640160916101709162018091B2
:102BB0006301909164012091FF02309100034091E4
:102BC0000103509102030E94254B1816C4F58CE3B3
:102BD00090E090938701809386018091F801909115
:102BE000F901009709F447C0209261013092620117
:102BF00040926301509264011092F9011092F80121
:102C00001092E0011092DF011092FB011092FA0184
:102C10000F900F900F900F90CF91DF911F910F9118
:102C2000FF90EF90DF90CF90BF90AF909F908F90EC
:102C30007F906F905F904F903F902F90089588E71E
:102C400090E090938701809386011092E0011092AA
:102C5000DF011092FB011092FA01DACF89819A818B
:102C6000AB81BC818093610190936201A093630169
:102C7000B093640198CF81E090E09093F901809344
:102C8000F801E3CFA0926101B0926201C0926301AA
:102C9000D09264010E94FE14909387018093860174
:102CA0009093E4018093E3018091DF019091E00132
:102CB0009093E2018093E1018091200380628093F0
:102CC00020031092E0011092DF0181E090E09093E8
:102CD000FB018093FA019CCFAF92BF92CF92DF921B
:102CE000EF92FF920F931F938091DA019091DB0195
:102CF000009721F5609113037091140380911503DF
:102D000090911603E0907901F0907A0100917B0197
:102D100010917C01A80197010E94D64987FF17C036
:102D20008091DC01882399F180918101882331F41D
:102D300088E790E09093DB018093DA011F910F9177
:102D4000FF90EF90DF90CF90BF90AF900895A0904C
:102D50001303B0901403C0901503D0901603C8015C
:102D6000B70120917D0130917E0140917F0150910A
:102D700080010E947249A60195010E94D64987FFF1
:102D8000DDCF1092DC018AE080938101D7CF809162
:102D90008101815080938101C9CF1F920F920FB69C
:102DA0000F920BB60F921124EF92FF920F931F9385
:102DB0002F933F934F935F936F937F938F939F9343
:102DC000AF93BF93EF93FF938091A9019091AA01D4
:102DD00001979093AA018093A901009709F001C17E
:102DE0006091FF02709100038091010390910203B2
:102DF0002091130330911403409115035091160351
:102E00000E94254B18160CF403C110E0409887E08F
:102E10000E94D90C209150013091510140915201F2
:102E2000509153010E94294B9B01AC012093130345
:102E300030931403409315035093160360911303CA
:102E400070911403809115039091160320E030E0F7
:102E500048ED51E40E94254B18169CF480919F0286
:102E60009091A002A091A102B091A2020196A11D91
:102E7000B11D80939F029093A002A093A102B093F2
:102E8000A20286E00E94D90C20914C0130914D01A4
:102E900040914E0150914F010E94294B9B01AC0182
:102EA0002093FF02309300034093010350930203E9
:102EB0006091FF02709100038091010390910203E1
:102EC00020E030E048ED51E40E94254B18169CF4B8
:102ED00080919B0290919C02A0919D02B0919E02D4
:102EE0000196A11DB11D80939B0290939C02A0931B
:102EF0009D02B0939E020E94A00D8091A00190912E
:102F0000A101A091A201B091A3010196A11DB11D43
:102F10008093A0019093A101A093A201B093A3017B
:102F2000112309F09CC0419A83E00E94D90C2091A2
:102F30005C0130915D0140915E0150915F010E9402
:102F4000294B2091C40123FF6EC020E030E040E215
:102F500050E40E9471492DEC3CEC4CEC5DE30E9486
:102F6000DA497B018C016E2D7F2D802F912F2091CE
:102F7000C5013091C6014091C7015091C8010E941E
:102F800071499B01AC0120939302309394024093CA
:102F9000950250939602409A85E00E94D90C2091A8
:102FA00054013091550140915601509157010E94B2
:102FB000294B9B01AC0120933102309332024093A4
:102FC0003302509334020E94F410A89585E090E0FB
:102FD0009093AA018093A90180912003816080933E
:102FE0002003FF91EF91BF91AF919F918F917F91BE
:102FF0006F915F914F913F912F911F910F91FF9092
:10300000EF900F900BBE0F900FBE0F901F90189572
:103010001092210210922202109223021092240296
:10302000419811E0F3CE20E030E040E05FE30E9401
:10303000714929EA37E848E05EE30E94DA497B01FA
:103040008C017F2D912F20E030E0A9010E94D6490C
:1030500087FF89CFEE24FF2400E010E084CF809129
:103060000F0390911003A0911103B091120380936C
:10307000390290933A02A0933B02B0933C0284E061
:103080000E94D90C209158013091590140915A0168
:1030900050915B010E94294B20E030E040E05FE36B
:1030A0000E94714929EA37E848E05EE30E94DA4964
:1030B0007B018C017F2D912F20E030E0A9010E943F
:1030C000D64987FF04C0EE24FF2400E010E06E2DF7
:1030D0007F2D802F912F2091C9013091CA014091FD
:1030E000CB015091CC010E9471499B01AC0120930E
:1030F0000F0330931003409311035093120313CF27
:10310000EF92FF920F931F9360910202709103025E
:10311000809104029091050220E030E0A9010E9414
:1031200072492091060230910702409108025091A5
:1031300009020E94724920910A0230910B024091CB
:103140000C0250910D020E94724920910E023091A2
:103150000F0240911002509111020E9472497B01AE
:103160008C0120911202309113024091140250916F
:103170001502CA01B9012E2D3F2D402F512F0E945B
:10318000724920E030E040EA50E40E94DA491F91A1
:103190000F91FF90EF900895A091CC028A2F65E0E7
:1031A0000E948C4BE92FF0E0209193023091940221
:1031B0004091950250919602EE0FFF1FEE0FFF1FF8
:1031C000EE5FFD4F2083318342835383AF5FA09333
:1031D000CC0280918A01882379F08091F501609179
:1031E0006001982F9F5F9093F5010E948C4B99236B
:1031F00019F481E08093D1010895AF92BF92CF92EC
:10320000DF92EF92FF920F931F938091F401982F1A
:103210009F5F9093F4016CE30E948C4B992309F417
:103220006AC18091D901882309F45AC18091C401EF
:103230008370833029F480914601882309F061C1AD
:1032400080918601909187010197909387018093E7
:1032500086018091DF019091E00101969093E00159
:103260008093DF016091CD017091CE018091CF01FB
:103270009091D00120E030E040E85FE30E94724985
:103280006093CD017093CE018093CF019093D001D4
:103290006091FF02709100038091010390910203FD
:1032A00020910F03309110034091110350911203AC
:1032B0000E94294B7B01082FB92E862F9F2DA02F0E
:1032C000BB2D80938B0290938C02A0938D02B093C0
:1032D0008E026E2D7F2D802F9B2D2091C802309164
:1032E000C9024091CA025091CB020E94254B181688
:1032F00064F48E2D9F2DA02FBB2D8093C802909338
:10330000C902A093CA02B093CB02609131027091BE
:1033100032028091330290913402209193023091D5
:10332000940240919502509196020E94294B162FCB
:10333000D72EC82EA92E862F9D2DAC2DBA2D809369
:10334000030390930403A0930503B0930603612F36
:103350007D2D8C2D9A2D2091350230913602409191
:103360003702509138020E94254B181664F4812FC1
:103370009D2DAC2DBA2D8093350290933602A093EB
:103380003702B09338026091160270911702809153
:103390001802909119022E2D3F2D402F5B2D0E9477
:1033A00072496093160270931702809318029093EB
:1033B00019026091070370910803809109039091AD
:1033C0000A03212F3D2D4C2D5A2D0E9472496093E6
:1033D0000703709308038093090390930A032091D5
:1033E0000F0330911003409111035091120360912B
:1033F00025027091260280912702909128020E9456
:10340000724960932502709326028093270290935D
:10341000280220919302309194024091950250919C
:10342000960260912D0270912E0280912F02909150
:1034300030020E94724960932D0270932E02809395
:103440002F02909330028091DA019091DB01009776
:1034500039F001979093DB018093DA01009721F115
:103460002091E5013091E60121153105A1F040E000
:1034700050E060919702709198028091990290912A
:103480009A020E94BF4B611571058105910519F4DF
:1034900081E08093E7011F910F91FF90EF90DF9003
:1034A000CF90BF90AF9008958091DC01882309F4FC
:1034B00047C081E08093DC018091AF029091B0021F
:1034C000A091B102B091B2020196A11DB11D8093ED
:1034D000AF029093B002A093B102B093B202C0CFFA
:1034E000609113037091140380911503909116035A
:1034F0000E9430159BCE81E08093F4010E94CC188D
:1035000090CE80914701882309F49ACE8091C20120
:10351000882309F095CE8091A80181508093A8015D
:10352000882309F08DCE81E08093C2010A9A129A15
:1035300083E08093A8018AE091E00E941F4F80CE33
:103540000E947612B6CF1F920F920FB60F920BB653
:103550000F9211242F933F934F935F936F937F9319
:103560008F939F93AF93BF93EF93FF93809120032B
:103570008260809320032091A601222341F480E100
:103580008093B2008091A7018F5F8093A701809103
:10359000880190918901181619067CF480918801A0
:1035A000909189010197909389018093880180917E
:1035B000880190918901009719F12223D1F080911F
:1035C000A70181508093A701882301F1FF91EF911A
:1035D000BF91AF919F918F917F916F915F914F912B
:1035E0003F912F910F900BBE0F900FBE0F901F9029
:1035F00018958091A701813149F71092A70109C060
:1036000080E00E9414122091A601D7CF80E1809320
:10361000A7018091970290919802A0919902B09190
:103620009A020196A11DB11D809397029093980272
:10363000A0939902B0939A020E9492440E94FD18AE
:103640008091210290912202A0912302B091240244
:103650000196A11DB11D8093210290932202A09397
:103660002302B09324028091DC01882309F4AECFB9
:103670008091290290912A02A0912B02B0912C02F4
:103680000196A11DB11D8093290290932A02A09357
:103690002B02B0932C029ACFCF93DF938EEA93E064
:1036A0002091AE033091AF03FC013197A081FC0162
:1036B00032977081FC0133976081FC01349750810F
:1036C0000597EC014881EDB7FEB73E970FB6F89429
:1036D000FEBF0FBEEDBF319684EF90E1CDB7DEB7F0
:1036E0009A83898333832283A48315827683178206
:1036F0006087118652871386448715860E94FF4E85
:10370000EDB7FEB73E960FB6F894FEBF0FBEEDBF05
:10371000DF91CF9108952F923F924F925F926F92D7
:103720007F928F929F92AF92BF92CF92DF92EF9251
:10373000FF920F931F93DF93CF93CDB7DEB72B97F5
:103740000FB6F894DEBF0FBECDBF009769F000D072
:1037500081EF90E1ADB7BEB712969C938E9311970F
:103760000E94FF4E0F900F90E0901303F09014030F
:1037700000911503109116032091610130916201AF
:1037800040916301509164018091FF029091000388
:10379000A0910103B09102038E839F83A887B9870C
:1037A000A0900F03B0901003C0901103D0901203AB
:1037B000A0919801B0919901BB87AA8760904801B8
:1037C0007090490180904A0190904B01B091DC01CA
:1037D000B9832090310230903202409033025090F1
:1037E00034028091930290919402A0919502B0913D
:1037F00096028A839B83AC83BD83ADB7BEB7969791
:103800000FB6F894BEBF0FBEADBFEDB7FEB7319691
:1038100061EB70E112967C936E931197E282F382D2
:103820000483158326833783408751878E819F8148
:10383000A885B98582879387A487B587A686B7862A
:10384000C08AD18AAA85BB85B38BA28B648A758A0C
:10385000868A978A8091DF019091E001918F808F15
:103860008091860190918701938F828FB981B48F67
:10387000158E268E378E40A251A28A819B81AC8103
:10388000BD8182A393A3A4A3B5A30E94FF4EADB7AD
:10389000BEB796960FB6F894BEBF0FBEADBF2B96BF
:1038A0000FB6F894DEBF0FBECDBFCF91DF911F9151
:1038B0000F91FF90EF90DF90CF90BF90AF909F90CF
:1038C0008F907F906F905F904F903F902F900895D2
:1038D0002F923F924F925F926F927F928F929F9220
:1038E000AF92BF92CF92DF92EF92FF920F931F930E
:1038F000DF93CF93CDB7DEB728970FB6F894DEBF2E
:103900000FBECDBFE090F201F090F3010894E11CEE
:10391000F11CF092F301E092F201C7018F709070F8
:10392000009789F4609148017091490180914A01A2
:1039300090914B0120E030E040E252E40E94254BA0
:1039400018160CF487C08091E701882309F09AC00B
:103950008091D2019091D30180FD6EC08091D201FF
:103960009091D30182FF09C08091F2019091F301FF
:103970008F709070009709F436C18091D2019091B8
:10398000D30183FF09C08091F2019091F3018F7000
:103990009070009709F472C18091D2019091D30187
:1039A00084FF04C08091200383FD0AC28091D2016C
:1039B0009091D30185FF04C08091200384FD40C213
:1039C0008091D2019091D30181FF04C080912003A6
:1039D00085FD76C28091D2019091D30181FF04C010
:1039E0008091200386FDE1C08091D2019091D301A6
:1039F00090FF09C08091F2019091F3018F70907057
:103A0000009709F44BC028960FB6F894DEBF0FBE9E
:103A1000CDBFCF91DF911F910F91FF90EF90DF907D
:103A2000CF90BF90AF909F908F907F906F905F905E
:103A30004F903F902F9008952FE0E222FF24E11451
:103A4000F10409F08BCF0E944C1B80E090E00E94B3
:103A50008B1B84CF8091B3029091B402A091B502E8
:103A6000B091B6020196A11DB11D8093B30290934F
:103A7000B402A093B502B093B6028091E701882307
:103A800009F466CF81E090E00E948B1B8091A40135
:103A9000882309F03FC21092E70160CF0E944C1BBF
:103AA000EDB7FEB77A970FB6F894FEBF0FBEEDBF25
:103AB000EDB6FEB60894E11CF11C86E79FE0928308
:103AC0008183609125027091260280912702909156
:103AD000280220E030E041E655E40E94DA49D701AF
:103AE00012966D937D938D939C93159760912D0203
:103AF00070912E0280912F029091300220E030E0F0
:103B000041E655E40E94DA49F701668377838087AE
:103B1000918780918B0290918C02A0918D02B0913F
:103B20008E0282879387A487B58780910303909143
:103B30000403A0910503B091060386879787A08BA5
:103B4000B18B6091160270911702809118029091CA
:103B5000190220E030E041E655E40E94DA49D7013D
:103B600052966D937D938D939C9355976091070327
:103B7000709108038091090390910A0320E030E0DE
:103B800041E655E40E94DA49F701668B778B808F16
:103B9000918F0E94FF4E2DB73EB7265E3F4F0FB666
:103BA000F8943EBF0FBE2DBF2ECF809120038F7B98
:103BB000809320038091E1019091E20100D000D038
:103BC00022EA3FE0ADB7BEB712963C932E93119711
:103BD00014969C938E9313970E94FF4E0F900F9014
:103BE0000F900F9001CF0E944C1BE0901303F090B8
:103BF00014030091150310911603209131023091A6
:103C000032024091330250913402A0909302B0905E
:103C10009402C0909502D090960280918C01909170
:103C20008D016DB77EB7605170400FB6F8947EBFBE
:103C30000FBE6DBFEDB7FEB7319666E970E1ADB767
:103C4000BEB712967C936E931197E282F38204833F
:103C500015832683378340875187A286B386C4861F
:103C6000D586978786870E94FF4EEDB7FEB7709680
:103C70000FB6F894FEBF0FBEEDBF7FCE0E944C1B67
:103C800020911303309114034091150350911603B2
:103C9000E0906101F0906201009163011091640174
:103CA0006090FF02709000038090010390900203E7
:103CB00020900F0330901003409011035090120396
:103CC00060919801709199017E836D8380918F023C
:103CD00090919002A0919102B091920289839A836F
:103CE000AB83BC8360918F027091900280919102AE
:103CF00090919202A0900B03B0900C03C0900D0322
:103D0000D0900E03ADB7BEB75E970FB6F894BEBFA6
:103D10000FBEADBFEDB7FEB73196F887EF83E0E693
:103D2000F0E11296FC93EE931197EF81F8852283D0
:103D3000338344835583AF81B8851696ED92FD9207
:103D40000D931C931997EF81F8856286738684869C
:103D50009586AF81B8851E962D923D924D925C92CC
:103D60005197ED81FE815396FC93EE9352972981F2
:103D70003A814B815C81AF81B88554962D933D93F8
:103D80004D935C93579720918A0158962C9358979E
:103D900059961C92A60195010E947149EF81F88500
:103DA000628F738F848F958F0E94FF4E2DB73EB721
:103DB000225E3F4F0FB6F8943EBF0FBE2DBFECCD35
:103DC0000E944C1B40913D0250913E022091C60240
:103DD0003091C7028091210390912203A091230387
:103DE000B09124036DB77EB76A5070400FB6F89457
:103DF0007EBF0FBE6DBFEDB6FEB60894E11CF11C90
:103E00006EE270E1EDB7FEB772836183F701538311
:103E100042833583248386839783A087B1870E945A
:103E2000FF4E80912003877F809320032DB73EB7FC
:103E3000265F3F4F0FB6F8943EBF0FBE2DBFB6CDE5
:103E40000E944C1B40913D0250913E022091C602BF
:103E50003091C7028091210390912203A091230306
:103E6000B09124036DB77EB76A5070400FB6F894D6
:103E70007EBF0FBE6DBFEDB6FEB60894E11CF11C0F
:103E800067EF7FE0EDB7FEB772836183F70153837D
:103E900042833583248386839783A087B1870E94DA
:103EA000FF4E809120038F7E809320032DB73EB775
:103EB000265F3F4F0FB6F8943EBF0FBE2DBF80CD9B
:103EC000809120038F7D809320032091E101309128
:103ED000E2018091E3019091E40100D000D000D094
:103EE000EDB7FEB7319645EC5FE0ADB7BEB71296C1
:103EF0005C934E93119733832283958384830E942E
:103F0000FF4EEDB7FEB736960FB6F894FEBF0FBE64
:103F1000EDBF60CD0E94FD43BECD0E946C16809126
:103F2000F0019091F10101969093F1018093F001DD
:103F30008F739070009709F491C06091FF027091A7
:103F400000038091010390910203209113033091AB
:103F5000140340911503509116030E94254B181627
:103F600034F482E090E0909389018093880160911D
:103F7000FF02709100038091010390910203209150
:103F800013033091140340911503509116030E94BE
:103F9000D64987FF09C08091F0019091F1018F7798
:103FA0009070009709F453C060911303709114034B
:103FB000809115039091160323E333E347E451E422
:103FC0000E94254B87FD09C08091F0019091F1017D
:103FD0008F779070009709F444C06091130370913B
:103FE000140380911503909116032DEC3CEC44E4EE
:103FF00051E40E94254B87FD08C08091F00190910B
:10400000F1018F7790700097B1F160911303709177
:104010001403809115039091160323EC35EF40E4CF
:1040200051E40E94254B87FD08C08091F0019091DA
:10403000F1018F779070009759F18091D2019091A2
:10404000D30187FF089581E00E941412089581E052
:1040500090E09093890180938801A6CF0E94CA13B3
:104060006CCF83E00E9414128091D2019091D30111
:1040700087FFE8CFE8CF83E00E94141282E00E941D
:1040800014128091D2019091D30187FFDBCFDBCF57
:1040900082E00E9414128091D2019091D30187FF97
:1040A000D1CFD1CF8091200380FD32C07894809110
:1040B000D4019091D5010097E9F08091A0019091F1
:1040C000A101A091A201B091A3010097A105B105A2
:1040D00089F48091940190919501A0919601B091FD
:1040E00097010097A105B10529F483B7817F866008
:1040F00083BF03C083B7817F83BFF89483B7816098
:1041000083BF7894889583B78E7F83BF7894089512
:10411000809120038E7F809320030E948D1FC6CF45
:104120000F931F93CF93DF9310E00E945344882393
:10413000A1F18091B0039091B1030E94914EEC01E6
:104140008FEFCF3FD80789F3CD30C9F0C231D10509
:1041500009F444C0CF37D10519F1C830D10501F1B8
:104160006091B2037091B303CE010E94D34EE12F50
:10417000F0E0E353FD4FC0831F5F1133B0F2212FF6
:1041800030E0F901E353FD4F10822F5F3F4FC9012B
:10419000DF91CF911F910F9108950E945220C5CFBA
:1041A000112311F410E0C1CF6091B2037091B303F9
:1041B00088E090E00E94D34E6091B2037091B30307
:1041C00080E290E00E94D34E6091B2037091B303FD
:1041D00088E090E00E94D34E1150CFCF6091B2039F
:1041E0007091B3038DE090E00E94D34E1123D1F281
:1041F000CDECD2E000E06091B2037091B3038991FD
:1042000090E00E94D34E0F5F0117A8F3B6CFEF9254
:10421000FF920F931F93CF93DF9300D089E691E134
:10422000EDB7FEB7928381830E94FF4E0F900F90EF
:104230008091B0039091B1030E949020823091054B
:1042400034F08091CD02893749F0893539F0DF911A
:10425000CF911F910F91FF90EF90089500D0CBEC7C
:10426000D1E1EDB7FEB7D283C1830E94FF4E8FE547
:1042700091E1EDB7FEB7928381830E94FF4EEDB7C7
:10428000FEB7D283C1830E94FF4E8FEF8093BB02A3
:104290008093BC028093BD028093BE028093BF02D4
:1042A0008093C0028093C1028093C2020F900F904E
:1042B0008BEB92E066E470E049E050E00E94C44F6E
:1042C0001092D90189ED91E065E370E041E050E0A2
:1042D0000E94C44F11E010938A018AE891E062E4E1
:1042E00070E041E050E00E94C44F10938B018BE8D6
:1042F00091E063E470E041E050E00E94C44F0F2E73
:10430000FEEAEF2EF7E4FF2EF1EE0F2FFCE31F2F56
:10431000F02DE0924C01F0924D0100934E0110936C
:104320004F018CE491E060E070E044E050E00E94D6
:10433000C44FE0925001F09251010093520110934A
:10434000530180E591E064E070E044E050E00E94B9
:10435000C44FE0925401F09255010093560110931E
:10436000570184E591E068E070E044E050E00E948D
:10437000C44F0F2EFAE0EF2EF7EDFF2EF3EA0F2FCA
:10438000FBE31F2FF02DE0925801F09259010093AA
:104390005A0110935B0188E591E06CE070E044E025
:1043A00050E00E94C44FE0925C01F0925D010093E6
:1043B0005E0110935F018CE591E060E170E044E004
:1043C00050E00E94C44F0F2EF0E0EF2EF0E0FF2EE1
:1043D000F0E00F2FF0E01F2FF02DE092C501F092DA
:1043E000C6010093C7011093C80185EC91E064E118
:1043F00070E044E050E00E94C44FE092C901F092A6
:10440000CA010093CB011093CC0189EC91E068E1E3
:1044100070E044E050E00E94C44F83E393E3A3E2E2
:10442000B1E48093610190936201A0936301B09322
:10443000640181E691E06DE170E044E050E00E94AB
:10444000C44F0F2EF0E0EF2EF0E0FF2EF8E50F2F17
:10445000F1E41F2FF02DE0926901F0926A010093C0
:104460006B0110936C0189E691E065E270E044E035
:1044700050E00E94C44F86E696E6A6E6B1E480933B
:104480006D0190936E01A0936F01B09370018DE662
:1044900091E069E270E044E050E00E94C44F80E0A7
:1044A00090E0AAE7B5E48093820190938301A09302
:1044B0008401B093850182E891E06EE370E044E00E
:1044C00050E00E94C44F80E090E0A0E9B1E4809306
:1044D000650190936601A0936701B093680185E63A
:1044E00091E061E270E044E050E00E94C44FE0924D
:1044F0006101F092620100936301109364010F2E39
:10450000F0E0EF2EF0E0FF2EF0EA0F2FF0E41F2F87
:10451000F02DE0927101F0927201009373011093FB
:10452000740181E791E06DE270E044E050E00E94A8
:10453000C44FE0927501F0927601009377011093D9
:10454000780185E791E061E370E044E050E00E948B
:10455000C44F80E090E0A0E4B1E4809379019093AF
:104560007A01A0937B01B0937C0189E791E066E337
:1045700070E044E050E00E94C44F8DEC9CECACE451
:10458000BFE380937D0190937E01A0937F01B09360
:1045900080018DE791E06AE370E044E050E00E9422
:1045A000C44F85E08093600180E691E06CE170E0AB
:1045B00041E050E00E94C44F1092E6011092E501E4
:1045C00085EE91E064E470E042E050E00E94C44F68
:1045D000DF91CF911F910F91FF90EF9008950E946E
:1045E0004C1B00D08BEC91E1EDB7FEB79283818339
:1045F0000E94FF4E0F900F90089587E59FE00E9464
:104600001D448CE19FE00E941D448091A6018823F7
:1046100089F183E191E000D000D024E13FE0EDB7E3
:10462000FEB732832183948383830E94FF4E80915F
:10463000BC030F900F900F900F9083FD1EC088E277
:1046400091E000D000D029E03FE0EDB7FEB7328323
:104650002183948383830E94FF4E0F900F908BECF5
:1046600091E1EDB7FEB7928381830E94FF4E0F90D8
:104670000F90089588E191E0CECF8FE191E0E1CFF6
:1046800083E09FE00E941D440895EF92FF920F93F4
:104690001F93CF93DF930E94FD2200D08DEF9EE009
:1046A000ADB7BEB712969C938E9311970E94FF4EA2
:1046B0000F900F900E94EF2200D085EF9EE0CDB7C3
:1046C000DEB79A8389830E94FF4E0F900F9060910E
:1046D0009702709198028091990290919A020E949B
:1046E000F20900D08BEE9EE0EDB7FEB79283818396
:1046F0000E94FF4E0F900F906091290270912A0244
:1047000080912B0290912C020E94F2098091D90194
:10471000882309F4EBC28091130390911403A091B4
:104720001503B091160300D000D000D025ED3EE077
:10473000CDB7DEB73A832983EDB7FEB78383948381
:10474000A583B6830E94FF4E2DB73EB72A5F3F4F29
:104750000FB6F8943EBF0FBE2DBF8091FF0290911F
:104760000003A0910103B091020300D000D000D05B
:104770002AEA3EE0CDB7DEB73A832983EDB7FEB72C
:1047800083839483A583B6830E94FF4E83E99EE0D2
:10479000ADB7BEB712969C938E93119780916D0121
:1047A00090916E01A0916F01B0917001CDB7DEB70D
:1047B0008B839C83AD83BE830E94FF4E8CE79EE07B
:1047C000EDB7FEB7928381838091690190916A0170
:1047D000A0916B01B0916C01CDB7DEB78B839C8348
:1047E000AD83BE830E94FF4E809161019091620172
:1047F000A0916301B091640126E63EE0EDB7FEB7FB
:1048000032832183CDB7DEB78B839C83AD83BE8398
:104810000E94FF4E8091310290913202A0913302AA
:10482000B09134022FE43EE0EDB7FEB7328321832E
:10483000CDB7DEB78B839C83AD83BE830E94FF4ED2
:1048400080910F0390911003A0911103B091120376
:104850002AE33EE0EDB7FEB732832183CDB7DEB762
:104860008B839C83AD83BE830E94FF4E8091930215
:1048700090919402A0919502B091960223E23EE0BD
:10488000EDB7FEB732832183CDB7DEB78B839C8330
:10489000AD83BE830E94FF4E87E09EE0EDB7FEB77A
:1048A000928381838091710190917201A091730133
:1048B000B0917401CDB7DEB78B839C83AD83BE838B
:1048C0000E94FF4E8CEE9DE0EDB7FEB79283818390
:1048D0008091750190917601A0917701B091780156
:1048E000CDB7DEB78B839C83AD83BE830E94FF4E22
:1048F0000F900F900F900F908FED9DE0EDB7FEB7EA
:10490000928381830E94FF4E0F900F90609121024D
:104910007091220280912302909124020E94F20958
:1049200000D000D000D08DEB9DE0ADB7BEB71296A1
:104930009C938E9311978091790190917A01A09127
:104940007B01B0917C01CDB7DEB78B839C83AD83B7
:10495000BE830E94FF4E8091DC01EDB7FEB7369614
:104960000FB6F894FEBF0FBEEDBF882309F0E4C177
:104970008091DD01882309F0D3C100D084E69DE059
:10498000EDB7FEB7928381830E94FF4E0F900F9088
:104990000E94371200D0CBECD1E1ADB7BEB7129672
:1049A000DC93CE9311970E94FF4E0F900F90809151
:1049B000DE01882309F0A8C100D000D000D08CE12E
:1049C0009DE0ADB7BEB712969C938E9311978091E0
:1049D0007D0190917E01A0917F01B0918001EDB7A2
:1049E000FEB783839483A583B6830E94FF4E2DB7C1
:1049F0003EB72A5F3F4F0FB6F8943EBF0FBE2DBFA4
:104A00008091D601882309F4BBC080914801909120
:104A10004901A0914A01B0914B0100D000D000D0D3
:104A200026E03DE0EDB7FEB7328321838383948394
:104A3000A583B6830E94FF4E2DB73EB72A5F3F4F36
:104A40000FB6F8943EBF0FBE2DBF8091BB028F3FC3
:104A500009F480C100D0EDB7FEB7D283C1830E94B4
:104A6000FF4E0F900F9080918A01882309F0C0C0FB
:104A700000D000D000D08AE09CE0CDB7DEB79A83AA
:104A800089838091650190916601A0916701B09141
:104A90006801EDB7FEB783839483A583B6830E9434
:104AA000FF4E609102027091030280910402909186
:104AB000050220E030E0A9010E947249209106021F
:104AC0003091070240910802509109020E947249F8
:104AD00020910A0230910B0240910C0250910D027C
:104AE0000E94724920910E0230910F0240911002F3
:104AF000509111020E9472497B018C012091120297
:104B0000309113024091140250911502CDB7DEB7D7
:104B10002196EBEEFBE0ADB7BEB71296FC93EE9399
:104B20001197CA01B9012E2D3F2D402F512F0E9400
:104B3000724920E030E040EA50E40E94DA496A839A
:104B40007B838C839D830E94FF4E0F900F9083ED9B
:104B50009BE0CDB7DEB79A8389838091E501909180
:104B6000E6019C838B830E94FF4E0F900F900F9065
:104B70000F90DF91CF911F910F91FF90EF900895CB
:104B800000D000D0EDB7FEB731968CEB9CE0ADB70E
:104B9000BEB712969C938E9311978091D701828312
:104BA00013820E94FF4E8091480190914901A0918B
:104BB0004A01B0914B0100D02BE93CE0CDB7DEB704
:104BC0003A832983EDB7FEB783839483A583B683A5
:104BD0000E94FF4E2DB73EB72A5F3F4F0FB6F894A5
:104BE0003EBF0FBE2DBF80918A01882309F440CFBC
:104BF0002091E8013091E9014091EA015091EB01E7
:104C00008091EC019091ED01A091EE01B091EF0146
:104C10006DB77EB76A5070400FB6F8947EBF0FBE76
:104C20006DBFEDB7FEB7319660E87CE0CDB7DEB77B
:104C30007A8369832283338344835583868397836E
:104C4000A087B1870E94FF4E20918B01EDB7FEB780
:104C50003A960FB6F894FEBF0FBEEDBF222309F0BF
:104C6000AAC040913D0250913E022091C60230916F
:104C7000C7028091210390912203A0912303B09158
:104C80002403CDB7DEB72A970FB6F894DEBF0FBE68
:104C9000CDBFEDB7FEB7319661E47CE07A836983DE
:104CA000538342833583248386839783A087B18788
:104CB0000E94FF4E20916001EDB7FEB736960FB609
:104CC000F894FEBF0FBEEDBF319685E29CE0ADB714
:104CD000BEB712969C938E931197228313820E94E3
:104CE000FF4E0F900F900F900F90C2CE8091130344
:104CF00090911403A0911503B091160300D000D039
:104D000000D02FEB3EE014CD00D084E49DE0EDB761
:104D1000FEB7928381830E94FF4E0F900F904CCE7E
:104D200000D08CE79DE0CDB7DEB79A8389830E94DF
:104D3000FF4E0F900F9021CE00D08BE99DE0ADB7D4
:104D4000BEB712969C938E9311970E94FF4E0F90C0
:104D50000F900ECE8091BC028F3F09F07BCE8091E8
:104D6000BD028F3F09F076CE8091BE028F3F09F0E1
:104D700071CE8091BF028F3F09F06CCE8091C0024E
:104D80008F3F09F067CE8091C1028F3F09F062CE5C
:104D90008091C2028F3F09F05DCE00D085ED9CE08E
:104DA000ADB7BEB712969C938E9311970E94FF4E9B
:104DB0000F900F904FCE00D000D0EDB7FEB73196D8
:104DC00080E79CE0ADB7BEB712969C938E93119787
:104DD000228313820E94FF4E0F900F900F900F902E
:104DE00040CFEF92FF920F931F93CF93DF93809169
:104DF000130390911403A0911503B091160300D0F2
:104E000000D000D02AEA3BE0EDB7FEB73283218321
:104E100083839483A583B6830E94FF4E8DB79EB78C
:104E200006960FB6F8949EBF0FBE8DBF8091B0035B
:104E30009091B1030E949020823050F18DEC92E06D
:104E40000E94264DE0901303F09014030091150387
:104E5000109116032091500130915101409152015F
:104E6000509153010E94294BA80197010E94DA49F1
:104E700060935001709351018093520190935301BC
:104E800080E591E064E070E044E050E00E94C44FAF
:104E900000D0CBECD1E1EDB7FEB7D283C1830E9445
:104EA000FF4E8091FF0290910003A0910103B09109
:104EB000020300D000D023E83BE0EDB7FEB7328319
:104EC000218383839483A583B6830E94FF4E8DB78D
:104ED0009EB706960FB6F8949EBF0FBE8DBF809109
:104EE000B0039091B1030E949020823050F18DEC7C
:104EF00092E00E94264DE090FF02F09000030091A6
:104F000001031091020320914C0130914D01409119
:104F10004E0150914F010E94294BA80197010E9418
:104F2000DA4960934C0170934D0180934E01909348
:104F30004F018CE491E060E070E044E050E00E94BA
:104F4000C44F00D0EDB7FEB7D283C1830E94FF4E9D
:104F50008091310290913202A0913302B0913402DB
:104F600000D000D02DE53BE0EDB7FEB732832183C2
:104F700083839483A583B6830E94FF4E8DB79EB72B
:104F800006960FB6F8949EBF0FBE8DBF8091B003FA
:104F90009091B1030E949020823050F18DEC92E00C
:104FA0000E94264DE0903102F090320200913302CF
:104FB00010913402209154013091550140915601D5
:104FC000509157010E94294BA80197010E94DA498C
:104FD000609354017093550180935601909357014B
:104FE00084E591E068E070E044E050E00E94C44F46
:104FF00000D0EDB7FEB7D283C1830E94FF4E8091EF
:10500000930290919402A0919502B091960200D0E3
:1050100000D027E33BE0EDB7FEB7328321838383E3
:105020009483A583B6830E94FF4E8DB79EB70696E4
:105030000FB6F8949EBF0FBE8DBF8091B0039091C4
:10504000B1030E949020823060F18DEC92E00E94CA
:10505000264D9B01AC016091930270919402809166
:105060009502909196020E9471499B01AC0160915A
:10507000C5017091C6018091C7019091C8010E943D
:1050800072496093C5017093C6018093C7019093E4
:10509000C80185EC91E064E170E044E050E00E94DA
:1050A000C44F00D0EDB7FEB7D283C1830E94FF4E3C
:1050B00080910F0390911003A0911103B0911203FE
:1050C00000D000D023E13BE0EDB7FEB7328321836F
:1050D00083839483A583B6830E94FF4E8DB79EB7CA
:1050E00006960FB6F8949EBF0FBE8DBF8091B00399
:1050F0009091B1030E949020823060F18DEC92E09B
:105100000E94264D9B01AC0160910F03709110032A
:1051100080911103909112030E9471499B01AC018F
:105120006091C9017091CA018091CB019091CC012D
:105130000E9472496093C9017093CA018093CB01A8
:105140009093CC0189EC91E068E170E044E050E09C
:105150000E94C44F00D0EDB7FEB7D283C1830E9436
:10516000FF4E0F900F90DF91CF911F910F91FF9005
:10517000EF900895CF93DF9300D000D000D08AEE57
:105180009AE0EDB7FEB79283818380916901909197
:105190006A01A0916B01B0916C0183839483A58314
:1051A000B6830E94FF4E8DB79EB706960FB6F89451
:1051B0009EBF0FBE8DBF8091B0039091B1030E943E
:1051C00090208230A0F08DEC92E00E94264D6093FA
:1051D000690170936A0180936B0190936C0189E679
:1051E00091E065E270E044E050E00E94C44F00D0DE
:1051F000CBECD1E1EDB7FEB7D283C1830E94FF4E65
:1052000000D000D081EC9AE0EDB7FEB792838183A5
:1052100080916D0190916E01A0916F01B09170012C
:1052200083839483A583B6830E94FF4E8DB79EB778
:1052300006960FB6F8949EBF0FBE8DBF8091B00347
:105240009091B1030E9490208230A0F08DEC92E00A
:105250000E94264D60936D0170936E0180936F01E3
:10526000909370018DE691E069E270E044E050E0D7
:105270000E94C44F00D0EDB7FEB7D283C1830E9415
:10528000FF4E8091690190916A01A0916B01B091EC
:105290006C018093610190936201A0936301B093CC
:1052A00064010F900F90DF91CF91089584EB9AE005
:1052B0000E941D4486EA9AE00E941D448AE89AE012
:1052C0000E941D448FE69AE00E941D448CE49AE0FF
:1052D0000E941D4480E39AE00E941D448AE09AE007
:1052E0000E941D448BEE99E00E941D4488EC99E0D9
:1052F0000E941D4483EB99E00E941D4487E999E0D8
:105300000E941D448DE799E00E941D4482E699E0C9
:105310000E941D448DE399E00E941D4483E299E0C0
:105320000E941D44089500D086E199E0EDB7FEB7D4
:10533000928381830E94FF4E8091A4010F900F9071
:10534000882309F408950E94FD43089589E099E0B7
:105350000E941D4481EF98E00E941D448AED98E070
:105360000E941D448CEC98E00E941D448AEB98E05A
:105370000E941D4485EA98E00E941D448AE898E056
:105380000E941D4489E798E00E941D448AE698E047
:105390000E941D448AE598E00E941D448CE398E039
:1053A0000E941D448BE198E00E941D448CEF97E021
:1053B0000E941D448AED97E00E941D448091C40123
:1053C00082FF17C08091C301882309F495C082E34E
:1053D00091E000D000D028EC37E0EDB7FEB7328383
:1053E0002183948383830E94FF4E0F900F900F9030
:1053F0000F9080918A01882309F075C08FE291E0B7
:1054000000D000D025EB37E0EDB7FEB73283218323
:10541000948383830E94FF4E0F900F900F900F9004
:1054200080918B01882309F05BC08FE291E000D06E
:1054300000D02AE937E0EDB7FEB7328321839483A9
:1054400083830E94FF4E0F900F908CE797E0EDB79B
:10545000FEB7928381830E94FF4E0F900F9088E6E3
:1054600097E00E941D4487E497E00E941D4488E273
:1054700097E00E941D448091C40180FF18C0809174
:1054800046018823B1F182E391E000D000D022E10F
:1054900037E0EDB7FEB732832183948383830E9484
:1054A000FF4E8091C4010F900F900F900F9081FFDD
:1054B00016C0809147018823C9F082E391E000D0B3
:1054C00000D025EF36E0EDB7FEB732832183948319
:1054D00083830E94FF4E0F900F900F900F900895BE
:1054E00082E391E0A4CF82E391E08ACF8FE291E062
:1054F000E6CF8FE291E0C9CF8FE291E06ACF2F92A1
:105500003F924F925F926F927F928F929F92AF9253
:10551000BF92CF92DF92EF92FF920F931F93CF93A0
:10552000DF93822E732E642E552E462E372E282E74
:10553000992E263609F48EC0282D372D462D552D4F
:10554000642D732D822D992D06E6A02E16E6B12E20
:10555000CC24DD24EE24FF2400E010E00E947F45EF
:105560008230E0F1882D893609F4ADC3282D372D1E
:10557000462D552D642D732D822D992DF9E6AF2ED4
:10558000E4E7BE2ECC24DD24EE24FF2400E010E06E
:105590000E947F45823008F0F1C0E82DE83609F41A
:1055A000D8C1882D853609F49BC1E82DE63709F46A
:1055B0004AC10E949329DF91CF911F910F91FF90D3
:1055C000EF90DF90CF90BF90AF909F908F907F90A3
:1055D0006F905F904F903F902F900895882D8C365C
:1055E00009F4DCC3282D372D462D552D642D732D40
:1055F000822D992DBCE6AB2EA1E6BA2ECC24DD245B
:10560000EE24FF2400E010E00E947F45823008F085
:105610008BC0E82DED3609F406C2F82DF93609F4F1
:10562000F9C2982D983629F6772019F6662009F6E2
:10563000552009F0BECF442009F0BBCF332009F03C
:10564000B8CF222009F0B5CF992009F0B2CF0E943F
:105650005629B1CF363609F06FCF442309F06CCF0D
:10566000552309F069CF662309F066CF772309F047
:1056700063CF882309F060CF992309F05DCF809133
:10568000A501882309F495CF00D08BE796E0EDB70C
:10569000FEB7928381830E94FF4E00D000D08DE53B
:1056A00096E0EDB7FEB7928381838091820190915D
:1056B0008301A0918401B091850183839483A583A4
:1056C000B6830E94FF4E8DB79EB706960FB6F8942C
:1056D0009EBF0FBE8DBF8091B0039091B1030E9419
:1056E000902082309105A4F08DEC92E00E94264D2E
:1056F000609382017093830180938401909385016C
:1057000082E891E06EE370E044E050E00E94C44F14
:1057100000D08BEC91E1EDB7FEB7928381830E94BC
:10572000FF4E0F900F9047CFE82DE13609F454C299
:10573000882D863709F4F7C1E82DE13609F039CF15
:10574000F72DF23609F035CF662009F032CF55201B
:1057500009F02FCF442009F02CCF332009F029CFB6
:10576000222009F026CF992009F023CF8091A501AE
:10577000882309F41ECF0E94BA281DCF882D8C36AD
:1057800009F478C1E82DE03709F467C1E82DE73660
:1057900009F00FCFF72DF63709F00BCF662009F08F
:1057A00008CF552009F005CF442009F002CF33205F
:1057B00009F0FFCE222009F0FCCE992009F0F9CEA5
:1057C0008091A501882309F4F4CE80916101909124
:1057D0006201A0916301B091640100D000D000D0BB
:1057E00023E436E0EDB7FEB73283218383839483CD
:1057F000A583B6830E94FF4E8DB79EB706960FB65F
:10580000F8949EBF0FBE8DBF8091B0039091B103FD
:105810000E949020823091050CF47ACF8DEC92E0BA
:105820000E94264D60936101709362018093630131
:105830009093640181E691E06DE170E044E050E016
:105840000E94C44F65CFF72DF63609F0B2CE662020
:1058500009F0AFCE552009F0ACCE442009F0A9CE16
:10586000332009F0A6CE222009F0A3CE992009F01A
:10587000A0CE81E09091D901911180E08093D9016F
:10588000882309F4E4C286E391E000D000D025ED3E
:1058900036E0EDB7FEB732832183948383830E9481
:1058A000FF4E0F900F900F900F908091D901882399
:1058B00009F0D0C289ED91E065E370E041E050E08D
:1058C0000E94C44F8091D901882309F474CE81E6E7
:1058D00091E06DE170E044E050E00E94B44F6BCE87
:1058E000972D943709F065CE662009F062CE5520D9
:1058F00009F05FCE442009F05CCE332009F059CE88
:10590000222009F056CE992009F053CE8091A501AE
:10591000882309F44ECE0E94CA13809148019091C9
:105920004901A0914A01B0914B0100D000D000D0B4
:105930002BE835E0EDB7FEB7328321838383948370
:10594000A583B6830E94FF4E0F900F900F900F908B
:10595000E0CEF72DF23709F02CCE662009F029CEE3
:10596000552009F026CE442009F023CE332009F03B
:1059700020CE222009F01DCE992009F01ACE809168
:10598000A501882309F415CE00D000D000D080EA0C
:1059900095E0EDB7FEB79283818380917D01909170
:1059A0007E01A0917F01B091800183839483A583C0
:1059B000B6830E94FF4E8DB79EB706960FB6F89439
:1059C0009EBF0FBE8DBF8091B0039091B1030E9426
:1059D0009020823091050CF49BCE60917D017091F6
:1059E0007E0180917F01909180012DEC3CEC4CEC8C
:1059F0005DE30E94254B18160CF08ACE8DEC92E0E8
:105A00000E94264D60937D0170937E0180937F01FB
:105A1000909380018DE791E06AE370E044E050E00C
:105A20000E94C44F75CE772009F0C3CD662009F0DF
:105A3000C0CD552009F0BDCD442009F0BACD3320AA
:105A400009F0B7CD222009F0B4CD992009F0B1CDED
:105A50001092D8010E94A629AECDF72DFC3609F090
:105A6000A8CD862D853609F0A4CD952D983609F060
:105A7000A0CDE1CD972D963709F09BCD662009F09A
:105A800098CD552009F095CD442009F092CD3320D2
:105A900009F08FCD222009F08CCD992009F089CD15
:105AA0008091A501882309F484CD00D000D000D0D6
:105AB00084E296E0EDB7FEB7928381838091650121
:105AC00090916601A0916701B091680183839483EE
:105AD000A583B6830E94FF4E8DB79EB706960FB67C
:105AE000F8949EBF0FBE8DBF8091B0039091B1031B
:105AF0000E949020823091050CF40ACE8DEC92E049
:105B00000E94264D60936501709366018093670142
:105B10009093680185E691E061E270E044E050E036
:105B20000E94C44FF5CD972D943609F042CD6620E2
:105B300009F03FCD552009F03CCD442009F039CD86
:105B4000332009F036CD222009F033CD992009F019
:105B500030CD8091A501882309F42BCD00D000D051
:105B600000D08EEB95E0EDB7FEB7928381838091F4
:105B7000790190917A01A0917B01B0917C0183839E
:105B80009483A583B6830E94FF4E8DB79EB7069679
:105B90000FB6F8949EBF0FBE8DBF8091B003909159
:105BA000B1030E949020823091050CF4B1CD8DECB0
:105BB00092E00E94264D6093790170937A01809360
:105BC0007B0190937C0189E791E066E370E044E01B
:105BD00050E00E94C44F9CCDF72DF33609F0B0CDB4
:105BE000662009F0E6CC552009F0E3CC442009F00A
:105BF000E0CC332009F0DDCC222009F0DACC99206A
:105C000009F0D7CC8091A501882309F4D2CC0E9459
:105C1000F126D1CC872D813609F0CBCC662009F056
:105C2000C8CC552009F0C5CC442009F0C2CC3320A3
:105C300009F0BFCC222009F0BCCC992009F0B9CCE6
:105C40008091A501882309F4B4CC00D000D000D005
:105C50008DEF95E0EDB7FEB792838183809171015E
:105C600090917201A0917301B09174018383948328
:105C7000A583B6830E94FF4E8DB79EB706960FB6DA
:105C8000F8949EBF0FBE8DBF8091B0039091B10379
:105C90000E949020823091050CF43ACD8DEC92E078
:105CA0000E94264D6093710170937201809373017D
:105CB0009093740181E791E06DE270E044E050E080
:105CC0000E94C44F25CD972D943709F04FCC662004
:105CD00009F04CCC552009F049CC442009F046CCC1
:105CE000332009F043CC222009F040CC992009F060
:105CF0003DCC8091A501882309F45BCC0E94710BF7
:105D000000D0CBECD1E1EDB7FEB7D283C1830E94C6
:105D1000FF4E8BE695E0EDB7FEB7928381830E943C
:105D2000FF4E0F900F908091B0039091B1030E94AD
:105D30009020823091053CF08DEC92E00E942A4D3B
:105D4000883008F4AFC000D0EDB7FEB7D283C1836E
:105D50000E94FF4E8AE495E0EDB7FEB792838183FF
:105D60000E94FF4E0F900F908091B0039091B1036D
:105D70000E949020823091053CF08DEC92E00E94D0
:105D80002A4D883008F472C000D0EDB7FEB7D28338
:105D9000C1830E94FF4E0F900F900DCC972D91362E
:105DA00009F020CC662009F01DCC552009F01ACC52
:105DB000442009F017CC332009F014CC222009F03C
:105DC00011CC992009F00ECC8091A501882309F40B
:105DD000F0CB00D000D000D087ED95E0EDB7FEB756
:105DE000928381838091750190917601A0917701D2
:105DF000B091780183839483A583B6830E94FF4E7C
:105E00008DB79EB706960FB6F8949EBF0FBE8DBF96
:105E10008091B0039091B1030E949020823091054F
:105E20000CF476CC8DEC92E00E94264D60937501C7
:105E300070937601809377019093780185E791E0E4
:105E400061E370E044E050E00E94C44F61CC89E31C
:105E500091E01BCD00D084EB96E0EDB7FEB79283C6
:105E600081830E94FF4E0F900F9024CD90E0FC01A3
:105E7000EE0FFF1FEE0FFF1FEE0FFF1FE80FF91FC2
:105E8000A7E1B3E0E15CFD4F89E001900D92815004
:105E9000E1F787E193E06FE470E049E050E00E94B1
:105EA000C44F72CF90E0FC01EE0FFF1FEE0FFF1FFB
:105EB000EE0FFF1FE80FF91FABEBB2E0E15CFD4F07
:105EC00089E001900D928150E1F78BEB92E066E45E
:105ED00070E049E050E00E94C44F35CF2F923F92CE
:105EE0004F925F926F927F928F929F92AF92BF92EA
:105EF000CF92DF92EF92FF920F931F93DF93CF9396
:105F0000CDB7DEB72C970FB6F894DEBF0FBECDBF6E
:105F1000822E732E642E552E462E372E282E992E25
:105F2000233709F446C1282D372D462D552D642DD4
:105F3000732D822D992D03E7A02E13E7B12ECC24CB
:105F4000DD24EE24FF2400E010E00E947F45823033
:105F500008F4D4C0282D213309F47FC5282D372D0E
:105F6000462D552D642D732D822D992DB1E3AB2E29
:105F7000A1E3BA2EF1E7CF2EDD24EE24FF2400E0CA
:105F800010E00E947F45823008F032C1782D7237D0
:105F900009F408C5282D372D462D552D642D732D58
:105FA000822D992DE2E7AE2E02E7B02E15E6C12E26
:105FB000DD24EE24FF2400E010E00E947F458230C3
:105FC00008F408C2F82DF53709F4A8C6682D603327
:105FD00009F033C1772D713309F02FC1862D813738
:105FE00009F02BC1552009F028C1442009F025C132
:105FF000332009F022C1222009F01FC1992009F0A5
:106000001CC100D08DE793E0ADB7BEB712969C934C
:106010008E9311970E94FF4EEDB7FEB77C970FB697
:10602000F894FEBF0FBEEDBF31968BE493E0ADB7A1
:10603000BEB712969C938E93119780919B0290917C
:106040009C02A0919D02B0919E0282839383A483BF
:10605000B58380919F029091A002A091A102B0917E
:10606000A20286839783A087B1878091A302909133
:10607000A402A091A502B091A60282879387A4876B
:10608000B5878091A7029091A802A091A902B09132
:10609000AA0286879787A08BB18B8091AB029091E3
:1060A000AC02A091AD02B091AE02828B938BA48B17
:1060B000B58B8091B3029091B402A091B502B091DA
:1060C000B602868B978BA08FB18F8091AF02909193
:1060D000B002A091B102B091B202828F938FA48FCF
:1060E000B58F0E94FF4EEDB7FEB77E960FB6F894BF
:1060F000FEBF0FBEEDBF21E030E0A1C0282D203350
:1061000009F485C4282D372D462D552D642D732D6A
:10611000822D992DB0E3AB2EA1E7BA2ECC24DD243D
:10612000EE24FF2400E010E00E947F45823008F05A
:10613000A0C0682D603709F4F0C3282D372D462DF7
:10614000552D642D732D822D992DF0E7AF2EECE6A1
:10615000BE2ECC24DD24EE24FF2400E010E00E94BB
:106160007F45823008F4B8C1A82DA93609F424C6A9
:10617000E82DE73709F061C0F72DFF3609F05DC063
:10618000662009F05AC0552009F057C0442009F094
:1061900054C0332009F051C0222009F04EC099208C
:1061A00009F04BC00E94710B8091A4018823E9F093
:1061B0004FC4333709F0B7CE442309F0B4CE55238A
:1061C00009F0B1CE662309F0AECE772309F0ABCE4D
:1061D000882309F0A8CE992309F0A5CE0E94452373
:1061E0008091A401882309F033C421E030E027C066
:1061F000982D943709F4EEC3282D372D462D552DB3
:10620000642D732D822D992DB4E7AB2EAFE6BA2EF7
:10621000FFE6CF2EE2E6DE2EEE24FF2400E010E0C3
:106220000E947F45823008F08AC0F82DF03709F4CB
:106230002BC5782D733709F4E1C420E030E0C901A3
:106240002C960FB6F894DEBF0FBECDBFCF91DF9175
:106250001F910F91FF90EF90DF90CF90BF90AF9084
:106260009F908F907F906F905F904F903F902F9076
:106270000895282D233309F4FBC2282D372D462DF0
:10628000552D642D732D822D992D03E3A02E11E73A
:10629000B12ECC24DD24EE24FF2400E010E00E9487
:1062A0007F45823008F40DC2A82DA43309F469C5D6
:1062B000E82DE03311F6F72DF23709F0BECF662056
:1062C00009F0BBCF552009F0B8CF442009F0B5CF75
:1062D000332009F0B2CF222009F0AFCF992009F086
:1062E000ACCF1092D3011092D2018091B003909163
:1062F000B1030E949020823091050CF4FDC58DEC15
:1063000092E00E94264D0E94424A8B018091B00388
:106310009091B1030E9490208230910554F08DEC51
:1063200092E00E94264D0E94424A0617170709F480
:106330000DC68091A401882309F457CF89C3B82DD5
:10634000B93609F492C5382D323709F076CF672D6A
:10635000673609F072CF762D703709F06ECF852D34
:10636000853709F06ACF442009F067CF332009F060
:1063700064CF222009F061CF992009F05ECF00D0D0
:1063800086E492E0ADB7BEB712969C938E931197B8
:106390000E94FF4E0F900F908091A4010E94FD4338
:1063A00088E10FB6F89480936000109260000FBEF1
:1063B00083ED9CE1FC01E115F10511F03197F1F756
:1063C0008115910511F00197F1F70C94007C21E003
:1063D00030E035CFA82DA83709F02FCFB72DB4372F
:1063E00009F02BCFE62DE13609F027CF552009F033
:1063F00024CF442009F021CF332009F01ECF2220E2
:1064000009F01BCF992009F018CF8091C40180FFBB
:10641000ABC381FFA9C380914701882309F490C5CC
:1064200086E391E000D000D023EB32E0ADB7BEB7F9
:1064300012963C932E93119714969C938E931397D8
:106440000E94FF4E809146010F900F900F900F9089
:10645000882309F472C586E391E000D000D023EAD6
:1064600032E0EDB7FEB732832183948383830E94A9
:10647000FF4E0F900F900F900F90019B5BC586E32E
:1064800091E000D000D02FE832E0ADB7BEB7129651
:106490003C932E93119714969C938E9313970E947E
:1064A000FF4E0F900F900F900F9002994CC522E471
:1064B00031E000D000D08BE792E0EDB7FEB79283D9
:1064C0008183348323830E94FF4E0F900F900F909F
:1064D0000F9021E030E0B3CE882D853609F0ADCEA7
:1064E000972D943609F0A9CE662009F0A6CE552046
:1064F00009F0A3CE442009F0A0CE332009F09DCEB0
:10650000222009F09ACE992009F097CE8091A5011A
:10651000882309F429C300D000D08DE395E0EDB7BE
:10652000FEB79283818381E090E0948383830E940D
:10653000FF4E8EE295E0ADB7BEB712969C938E9358
:10654000119782E090E014969C938E9313970E948B
:10655000FF4E81E295E0EDB7FEB79283818384E040
:1065600090E0948383830E94FF4E84E195E0ADB771
:10657000BEB712969C938E93119788E090E0149684
:106580009C938E9313970E94FF4E82E095E0EDB7A7
:10659000FEB79283818380E190E0948383830E949D
:1065A000FF4E8BEE94E0ADB7BEB712969C938E93E0
:1065B000119780E290E014969C938E9313970E941B
:1065C000FF4E80EE94E0EDB7FEB79283818380E4C6
:1065D00090E0948383830E94FF4E84ED94E0ADB7F6
:1065E000BEB712969C938E93119780E890E0149614
:1065F0009C938E9313970E94FF4E86EC94E0EDB728
:10660000FEB79283818380E091E0948383830E942C
:10661000FF4E8091D2019091D3012CEA34E0ADB7C6
:10662000BEB712963C932E93119714969C938E931B
:1066300013970E94FF4E0F900F900F900F90809134
:10664000B0039091B1030E9490208230910564F0D4
:106650008DEC92E060E070E040E150E00E94184C68
:106660007093D3016093D20100D08BEC91E1EDB730
:10667000FEB7928381830E94FF4E8091D201909158
:10668000D3010F900F9080FD72C48091D201909140
:10669000D30190FD60C48091D2019091D30183FF1A
:1066A000A4CD00D088EC93E0ADB7BEB712969C9312
:1066B0008E9311970E94FF4E0F900F9021E030E0D3
:1066C000BECD682D613309F441C3882D823309F0B2
:1066D000B4CD972D913709F0B0CD662009F0ADCD3E
:1066E000552009F0AACD442009F0A7CD332009F0A8
:1066F000A4CD222009F0A1CD992009F09ECD1092C1
:10670000D3011092D2018090130390901403A090B3
:106710001503B09016032091610130916201409100
:106720006301509164016091FF02709100038091B8
:1067300001039091020369877A878B879C87409039
:106740000F03509010036090110370901203E090BB
:106750004801F090490100914A0110914B0130909D
:10676000DC018091310290913202A0913302B0910C
:10677000340289839A83AB83BC83609193027091C6
:10678000940280919502909196026D837E838F830F
:1067900098878DB79EB78C970FB6F8949EBF0FBEA3
:1067A0008DBFEDB7FEB7319666EC71E0ADB7BEB701
:1067B00012967C936E93119782829382A482B58203
:1067C000268337834087518769857A858B859C85A9
:1067D000628773878487958746865786608A718A21
:1067E000E28AF38A048B158B8091790190917A016A
:1067F000A0917B01B0917C01868B978BA08FB18F8C
:1068000080917D0190917E01A0917F01B0918001E6
:10681000828F938FA48FB58F8091DD01868F178E25
:1068200030A211A28091DA019091DB0193A382A39F
:1068300089819A81AB81BC8184A395A3A6A3B7A3C8
:106840006D817E818F81988560A771A782A793A7AC
:106850000E94FF4E8091A401ADB7BEB79C960FB6C3
:10686000F894BEBF0FBEADBF882309F4BECCF0C004
:10687000372D313709F001CD662009F0FECC5520C7
:1068800009F0FBCC442009F0F8CC332009F0F5CC1A
:10689000222009F0F2CC992009F0EFCC1092D3011C
:1068A0001092D201209113033091140340911503EB
:1068B000509116038091930290919402A0919502B9
:1068C000B0919602EDB7FEB73A970FB6F894FEBFB7
:1068D0000FBEEDBFEDB6FEB60894E11CF11C67EBF0
:1068E00071E072836183F70122833383448355838C
:1068F00086839783A087B1870E94FF4E8091A40171
:106900002DB73EB7265F3F4F0FB6F8943EBF0FBE80
:106910002DBF882309F469CC9BC0772D7C3609F004
:106920000CCC662009F009CC552009F006CC442097
:1069300009F003CC332009F000CC222009F0FDCB74
:10694000992009F0FACB8091C40182FF0DC190918A
:10695000C30181E0911180E08093C3018091C30164
:10696000882309F4DAC226E331E000D000D08EE0BB
:1069700092E0ADB7BEB712969C938E931197149682
:106980003C932E9313970E94FF4E8091C3010F906A
:106990000F900F900F90882309F4BBC25F9A21E0FB
:1069A00030E04DCC872D823709F0F4CA962D95360C
:1069B00009F0F0CA552009F0EDCA442009F0EACAEE
:1069C000332009F0E7CA222009F0E4CA992009F42B
:1069D00018CBE0CAA72DAF3609F00ECCB62DBF36C6
:1069E00009F00ACCE52DE23609F006CC442009F086
:1069F00003CC332009F000CC222009F0FDCB9920F4
:106A000009F0FACB0C94000021E030E018CC372DCF
:106A1000313709F077CB662009F074CB552009F0A7
:106A200071CB442009F06ECB332009F06BCB2220D0
:106A300009F068CB992009F065CB1092D301109230
:106A4000D2010E9440238091A401882309F4CDCB78
:106A50000E94FD4321E030E0F2CB372D313309F0C5
:106A60007DCA662D613709F079CA552009F076CACA
:106A7000442009F073CA332009F070CA222009F0BB
:106A80006DCA992009F06ACAF89449E021E030E023
:106A9000F90140935700C895E02C20E030E0F9015F
:106AA00040935700C895902C7894F89423E030E0F8
:106AB000F90140935700C895802C82E090E0FC01DA
:106AC00040935700C895702C789400D000D000D027
:106AD00041E453E0ADB7BEB712965C934E93119765
:106AE0008091870290918802A0918902B0918A02D8
:106AF000EDB7FEB783839483A583B6830E94FF4ED0
:106B000000D000D0EDB7FEB731964AE153E0ADB703
:106B1000BEB712965C934E93119772821382848251
:106B2000158296821782E08611860E94FF4EEDB78D
:106B3000FEB73A960FB6F894FEBF0FBEEDBFEDEB71
:106B4000F3E020E4EF3FF20709F098F480E090E0F2
:106B500005C030E4EF3FF30709F068F43196208177
:106B6000253CB9F70196F5CF0E94932921E030E04A
:106B700066CB80E090E000D000D028E033E0ADB7F5
:106B8000BEB712963C932E93119714969C938E93B6
:106B900013970E94FF4E20916600EDB7FEB7319625
:106BA0008CEF92E0ADB7BEB712969C938E9311977F
:106BB000228313820E94FF4E8091C4009091C500F1
:106BC00021EF32E0EDB7FEB73283218394838383D4
:106BD0000E94FF4E0F900F908BEC91E1ADB7BEB7C6
:106BE00012969C938E9311970E94FF4E8091A40160
:106BF0000F900F90882309F4F8CA2ACF872D883781
:106C000009F01BCB962D943709F017CBA52DA13693
:106C100009F013CB442009F010CB332009F00DCB41
:106C2000222009F00ACB992009F007CB8091C401FA
:106C300081FF9ACF9091470181E0911180E080938C
:106C4000470180914701882309F460C126E331E0C0
:106C500000D000D08AE492E0EDB7FEB79283818342
:106C6000348323830E94FF4E809147010F900F9041
:106C70000F900F90882309F442C181E090E00E94B8
:106C8000960A21E030E0DBCA272D283709F0D5CA63
:106C9000362D343709F0D1CA652D613609F0CDCAD9
:106CA000442009F0CACA332009F0C7CA222009F0DB
:106CB000C4CA992009F0C1CA8091C40180FF54CF91
:106CC0009091460181E0911180E08093460180918E
:106CD0004601882309F42BC126E331E000D000D01F
:106CE00084E692E0ADB7BEB712969C938E9311974F
:106CF00014963C932E9313970E94FF4E8091460169
:106D00000F900F900F900F90882309F409C181E034
:106D100090E00E94850A21E030E091CA272D2336B9
:106D200009F08BCA362D3D3609F087CA552009F087
:106D300084CA442009F081CA332009F07ECA222087
:106D400009F07BCA992009F078CA9ECE772D713759
:106D500009F073CA662009F070CA552009F06DCA9F
:106D6000442009F06ACA332009F067CA222009F0DA
:106D700064CA992009F061CA1092D3011092D2011D
:106D80002DCAB72DB13709F058CA662009F055CA87
:106D9000552009F052CA442009F04FCA332009F0A7
:106DA0004CCA222009F049CA992009F046CA10921B
:106DB000D3011092D201F6C9B72DBD3609F03DCAF4
:106DC000662009F03ACA552009F037CA442009F074
:106DD00034CA332009F031CA222009F02ECA992082
:106DE00009F02BCA8091A501882309F4BDCE20911A
:106DF000600100D000D0EDB7FEB731968FE192E090
:106E0000ADB7BEB712969C938E93119722831382CF
:106E10000E94FF4E0F900F900F900F908091B00343
:106E20009091B1030E9490208230910584F08DEC06
:106E300092E00E94264D0E94474A6093600180E6DE
:106E400091E06CE170E041E050E00E94C44F00D05E
:106E50008BEC91E1EDB7FEB7928381830E94FF4EE8
:106E60000F900F9021E030E0EAC9E72DE33609F0FA
:106E7000E4C9F62DF33709F0E0C9252D2F3609F0C6
:106E8000DCC9442009F0D9C9332009F0D6C9222031
:106E900009F0D3C9992009F0D0C98091A5018823B0
:106EA00009F462CE2091660000D000D0EDB7FEB7A5
:106EB000319683EC92E0ADB7BEB712969C938E9359
:106EC0001197228313820E94FF4E0F900F900F9014
:106ED0000F908091B0039091B1030E949020823076
:106EE00091050CF4B4CF8DEC92E00E94264D0E94E7
:106EF000474A60936600ABCF0FEF1FEF07CA80E0F1
:106F000090E00E94960A21E030E099C929E331E03F
:106F10009FCE5F9821E030E092C929E331E025CD92
:106F200080E090E00E94850A21E030E088C929E3F2
:106F300031E0D4CE89E391E0A4CA89E391E08DCA1F
:106F400089E391E06FCA2DE331E0B3CA1093DB010E
:106F50000093DA01EEC900D084E194E0EDB7FEB70A
:106F6000928381830E94FF4E0F900F9094CB00D0AC
:106F70008BE594E0ADB7BEB712969C938E931197B4
:106F80000E94FF4E0F900F9080CB0F931F93CF93D3
:106F9000DF9300D000D000D087E791E0EDB7FEB7D7
:106FA000928381838091CD019091CE01A091CF01F8
:106FB000B091D00183839483A583B6830E94FF4E52
:106FC0000F900F900F900F900BEC11E1EDB7FEB703
:106FD000128301830E94FF4E8DB79EB740970FB674
:106FE000F8949EBF0FBE8DBFCDB7DEB721968FE45C
:106FF00091E0EDB7FEB79283818360912502709195
:107000002602809127029091280220E030E041E69C
:1070100055E40E94DA496A837B838C839D83809147
:107020008B0290918C02A0918D02B0918E028E8382
:107030009F83A887B9878091C8029091C902A091C7
:10704000CA02B091CB028A879B87AC87BD876091CB
:10705000160270911702809118029091190220E097
:1070600030E041E655E40E94DA496E877F87888BDD
:10707000998B0E94FF4E8DB79EB740960FB6F8943D
:107080009EBF0FBE8DBFEDB7FEB7128301830E9476
:10709000FF4E8DB79EB740970FB6F8949EBF0FBEB8
:1070A0008DBFCDB7DEB7219687E291E0EDB7FEB791
:1070B0009283818360912D0270912E0280912F0224
:1070C0009091300220E030E041E655E40E94DA4938
:1070D0006A837B838C839D83809103039091040357
:1070E000A0910503B09106038E839F83A887B9877B
:1070F0008091350290913602A0913702B09138020A
:107100008A879B87AC87BD876091070370910803CE
:107110008091090390910A0320E030E041E655E4B4
:107120000E94DA496E877F87888B998B0E94FF4E79
:107130008DB79EB740960FB6F8949EBF0FBE8DBF19
:10714000EDB7FEB7128301830E94FF4E0F900F90A0
:10715000DF91CF911F910F910895F89491E2E0E0B3
:10716000F0E0909357008491E2E0F0E090935700B4
:107170002491E4E0F0E090935700E49190E0A0E0E7
:10718000B0E0DC019927882730E040E050E0542F40
:10719000432F322F2227820F931FA41FB51F8E0F5C
:1071A000911DA11DB11D8093870290938802A09329
:1071B0008902B0938A02789408952F923F924F9259
:1071C0005F926F927F928F929F92AF92BF92CF9277
:1071D000DF92EF92FF920F931F93DF93CF93CDB780
:1071E000DEB760970FB6F894DEBF0FBECDBF80E864
:1071F0008093610082E0809361000E94AD388091AD
:10720000870290918802A0918902B0918A0285300C
:1072100027E992072EE1A20720E0B20709F435C75B
:1072200084E690E09093E0018093DF010E94C81211
:1072300081E00E9414120E9485448EE394E46DE67E
:1072400074E40E94464E02C00E9459440E94534476
:107250008823D1F70E94CA130E94FD228091D90190
:10726000882341F5209148013091490140914A011C
:1072700050914B0160E070E080EA91E40E94714916
:1072800026EA3BE944EC5CE30E94294B209169012A
:1072900030916A0140916B0150916C010E947249DA
:1072A0009B01AC0120936101309362014093630123
:1072B000509364018091200381FD12C080E090E032
:1072C0007C0108C00894E11CF11CF5E6EF16F104FE
:1072D00009F4E1C60E9452208091200381FFF2CF81
:1072E0002BEC31E18CEF90E09C838B83A5EEB0E03A
:1072F000BE83AD83EAECF0E0F887EF838AEA90E0A2
:107300009A878987ABE9B0E0BC87AB87ECE8F0E00F
:10731000FE87ED87388B2F8702C00E945220809114
:10732000200381FFFACF809120038D7F809320037B
:107330000E94681C0E945344882379F38091B00313
:107340009091B1030E9490208130910509F4FAC018
:107350008230910509F479C08330910509F4DCC0CD
:107360008430910509F4F7C08530910509F45FC2B6
:10737000AAE02A2E33244424552466247724882422
:10738000992400D0EF85F889ADB7BEB71296FC936B
:10739000EE9311970E94FF4E0F900F909101A20162
:1073A000B301C4010E946E2F009709F0B6CF8091FF
:1073B000D801813009F430C3F22DF33709F465C1E7
:1073C0009101A201B301C401F3E7AF2EE3E6BE2EA3
:1073D000CC24DD24EE24FF2400E010E00E947F4551
:1073E0008230E0F5322D353709F472C39101A201E4
:1073F000B301C40105E7A02EBB24CC24DD24EE2478
:10740000FF2400E010E00E947F45823008F0D4C1E4
:10741000822D823609F435C49101A201B301C40161
:1074200012E6A12EBB24CC24DD24EE24FF2400E0B0
:1074300010E00E947F45823008F06FC3922D913694
:1074400009F478C50E94932968CF2090CD02332497
:107450004424552466247724430193CFF22DF93632
:1074600009F4E1C29101A201B301C401F9E6AF2E12
:10747000E2E7BE2ECC24DD24EE24FF2400E010E061
:107480000E947F45823008F020C1322D3D3609F43C
:10749000ADC49101A201B301C4010DE6A02E15E611
:1074A000B12ECC24DD24EE24FF2400E010E00E9465
:1074B0007F45823008F081C3922D993609F4AFC51B
:1074C000B22DBC3609F0BECFE32DE43609F0BACFB9
:1074D000442009F0B7CF552009F0B4CF662009F059
:1074E000B1CF772009F0AECF882009F0ABCF99203B
:1074F00009F0A8CF8091A501882309F4A3CFF1E07A
:10750000F093DD010E9476128091A401882309F492
:1075100004CF0E94FD4301CFF091CD02FA8319827E
:107520008091CE0229813A81280F311DC9011901AC
:10753000892F880F880B482E582E682E782E882E7B
:10754000982E1FCF6091B2037091B3038AE090E050
:107550000E94D34EE2CE2091CD0230E040E050E0D8
:1075600060E070E080E090E000E10E940E45122FA4
:10757000F32EE42ED52EC62EB72EA82E292E20911E
:10758000CE0230E040E050E060E070E080E090E06B
:1075900008E00E940E45210FF1E0211708F0F0E00D
:1075A0003F0DE1E03F1508F0E0E0F30FA1E0F31735
:1075B00008F0A0E0EA2B4E0D31E04E1508F030E067
:1075C000E40FA1E0E41708F0A0E03A2B5D0DA1E084
:1075D0005D1508F0A0E0350F41E0351708F040E0F8
:1075E000A42B6C0D51E06C1508F050E0A60F41E0A3
:1075F000A61708F040E0542B7B0D41E07B1508F006
:1076000040E0570F61E0571708F060E0462B8A0D05
:1076100061E08A1508F060E0480F71E0481708F053
:1076200070E0672B920D960F8091CF02820F61E080
:10763000821708F060E06F0F71E06F1708F070E0DC
:107640007E0F21E07E1708F020E0E22FE30F21E01B
:10765000E31708F020E0322F3A0FF1E03A1708F074
:10766000F0E0F50F21E0F51708F020E0240F51E0DD
:10767000241708F050E0282E362E472E5E2E632E5B
:107680007F2E822E952E990E7CCE232D233609F047
:1076900097CE442009F094CE552009F091CE662073
:1076A00009F08ECE772009F08BCE882009F088CEA5
:1076B000992009F085CE0E94C5378091A4018823C6
:1076C00009F42BCE0E94FD4328CE922D953609F465
:1076D00074C39101A201B301C401B5E6AB2EA4E7C6
:1076E000BA2EF1E6CF2EE4E6DE2EEE24FF2400E0F3
:1076F00010E00E947F45823008F0AEC2F22DF337D1
:1077000009F436C4322D333709F09CCE832D8437EB
:1077100009F098CE442009F095CE552009F092CE7C
:10772000662009F08FCE772009F08CCE882009F0F2
:1077300089CE992009F086CE8091B0039091B10353
:107740000E949020803191050CF488C4F8948DEC4F
:1077500092E00E942A4D9093AF038093AE0382ED96
:1077600092E00E942A4D8093AD0385ED92E00E9445
:107770002A4D8093AC0388ED92E00E942A4D8093BD
:10778000AB038BED92E00E942A4D8093AA038EED0D
:1077900092E00E942A4D8093A903789400D0EF854F
:1077A000F889ADB7BEB71296FC93EE9311970E947D
:1077B000FF4E0F900F9081CFE22DE33609F47FC288
:1077C0009101A201B301C401B3E6AB2EA3E6BA2E28
:1077D000CC24DD24EE24FF2400E010E00E947F454D
:1077E000823008F0BFC1222D263709F44BC3322D59
:1077F0003D3609F027CE832D823609F023CE442072
:1078000009F020CE552009F01DCE662009F01ACED1
:10781000772009F017CE882009F014CE992009F0BE
:1078200011CEB1E0B093D8010E94562976CD2091B7
:10783000CD0230E040E050E060E070E080E090E0B9
:1078400008E10E940E45122FF32EE42ED52EC62EEF
:10785000B72EA82E292E2091CE0230E040E050E035
:1078600060E070E080E090E000E10E940E45210FB2
:10787000F1E0211708F0F0E03F0DE1E03F1508F0DE
:10788000E0E0F30FA1E0F31708F0A0E0EA2B4E0DC3
:1078900031E04E1508F030E0E40FA1E0E41708F005
:1078A000A0E03A2B5D0D41E05D1508F040E0350F9A
:1078B000A1E0351708F0A0E04A2B6C0D51E06C15E3
:1078C00008F050E0460FA1E0461708F0A0E05A2B60
:1078D0007B0D61E07B1508F060E0570FA1E05717C2
:1078E00008F0A0E06A2B8A0D71E08A1508F070E0BC
:1078F000680FA1E0681708F0A0E07A2B920D970FAF
:107900001091D002120F81E0121708F080E0F82EDB
:10791000FF0E81E0FF1608F080E0E82EEE0E81E019
:10792000EE1608F080E0D82ED30E81E0D31608F0D2
:1079300080E0C82EC40E81E0C41608F080E0B82EA6
:10794000B50E81E0B51608F080E0A82EA60E81E005
:10795000A61608F080E0282E290E2091CF0230E0F4
:1079600040E050E060E070E080E090E008E00E94DD
:107970000E45210FE1E0211708F0E0E0FF2DF30FA5
:1079800031E0FF1508F030E0EF0FA1E0EF1708F04D
:10799000A0E03A2B4E0DF1E04E1508F0F0E0340F68
:1079A000A1E0341708F0A0E0FA2B5D0D41E05D1571
:1079B00008F040E0F50FA1E0F51708F0A0E04A2B31
:1079C0006C0D51E06C1508F050E0460FA1E0461731
:1079D00008F0A0E05A2B6B2D670F71E06B1508F0D3
:1079E00070E0560FA1E0561708F0A0E07A2B8A0D40
:1079F00061E08A1508F060E0780FA1E0781708F0E0
:107A0000A0E06A2B920D222E3E2E432E5F2E3A01CD
:107A1000872E962E990EB5CC9101A201B301C40117
:107A20000E947F2A7ACC232D223709F01BCD4420D7
:107A300009F018CD552009F015CD662009F012CDBA
:107A4000772009F00FCD882009F00CCD992009F09E
:107A500009CD00D000D0E985FA85ADB7BEB7129642
:107A6000FC93EE9311978091E5019091E6011496B5
:107A70009C938E9313970E94FF4E0F900F900F9040
:107A80000F908091B0039091B1030E9490208230BA
:107A9000910584F08DEC92E00E942A4D9093E601CE
:107AA0008093E50185EE91E064E470E042E050E00F
:107AB0000E94C44F00D0EF85F889ADB7BEB71296CB
:107AC000FC93EE9311970E94FF4E0F900F9025CCE0
:107AD000332009F08BCC442009F088CC552009F0E4
:107AE00085CC662009F082CC772009F07FCC8820F5
:107AF00009F07CCC992009F079CC609197027091C3
:107B000098028091990290919A020E94F2098091C4
:107B1000A401882309F401CCFCCCA22DA83609F4D9
:107B200040C2B22DB43709F08DCC332009F08ACC95
:107B3000442009F087CC552009F084CC662009F058
:107B400081CC772009F07ECC882009F07BCC99206D
:107B500009F078CC0E94EF228091A401882309F4D7
:107B6000DCCBD7CC922D993609F433C2B22DBC367A
:107B700009F068CCE32DE33609F064CC442009F029
:107B800061CC552009F05ECC662009F05BCC7720F3
:107B900009F058CC882009F055CC992009F052CC36
:107BA0008091A501882309F44DCC1092DD018091CC
:107BB000A401882309F4B1CBACCCF22DF23609F440
:107BC0007EC1322D343709F03DCC832D8D3609F03E
:107BD00039CC442009F036CC552009F033CC66204E
:107BE00009F030CC772009F02DCC882009F02ACC80
:107BF000992009F027CC81E090918A01911180E0D1
:107C000080938A01882309F43DC231E03093D10189
:107C100086E391E000D000D0ED81FE81ADB7BEB724
:107C20001296FC93EE93119714969C938E93139750
:107C30000E94FF4E0F900F900F900F908AE891E0F6
:107C400062E470E041E050E00E94C44F8091A401E2
:107C5000882309F462CB5DCC922D903709F4F9C0EA
:107C6000F22DF43709F0EECB232D203709F0EACBC3
:107C7000342D303709F0E6CB852D8D3609F0E2CB77
:107C8000AECF332009F0C8CB442009F0C5CB552036
:107C900009F0C2CB662009F0BFCB772009F0BCCB3E
:107CA000882009F0B9CB992009F0B6CB81E090E0AB
:107CB0000E94BC0988B1A1E08A2788B92ECBF32D98
:107CC000F33609F07DCD442009F07ACD552009F036
:107CD00077CD662009F074CD772009F071CD88202A
:107CE00009F06ECD992009F06BCD00D0ED85FE85B1
:107CF000ADB7BEB71296FC93EE9311970E94FF4E5C
:107D0000EF85F889ADB7BEB71296FC93EE93119745
:107D10000E94FF4E80E090E0DC0180931602909379
:107D20001702A0931802B09319028093C80290938F
:107D3000C902A093CA02B093CB0280938B029093A6
:107D40008C02A0938D02B0938E02809325029093B3
:107D50002602A0932702B0932802809307039093F2
:107D60000803A0930903B0930A038093350290930C
:107D70003602A0933702B0933802809303039093A6
:107D80000403A0930503B093060380932D02909300
:107D90002E02A0932F02B09330028093CD019093D6
:107DA000CE01A093CF01B093D0018091A4010F9098
:107DB0000F90882309F4B1CAACCBA32DA43709F0E6
:107DC00088CCB42DB13609F084CCE52DE43609F029
:107DD00080CC662009F07DCC772009F07ACC882011
:107DE00009F077CC992009F4B5CE73CC832D853674
:107DF00009F04FCB442009F04CCB552009F049CB7A
:107E0000662009F046CB772009F043CB882009F0A3
:107E100040CB992009F03DCB81E09091A5019111D3
:107E200080E08093A501882309F429C186E391E0CD
:107E300000D000D02B813C81EDB7FEB73283218387
:107E4000948383830E94FF4E0F900F900F900F90AA
:107E500064CAA32DAC3609F003CFB42DB53609F0B2
:107E6000FFCEE52DE83609F0FBCE662009F0F8CE0E
:107E7000772009F0F5CE882009F0F2CE992009F498
:107E8000A5C0EECE332009F0B2CC442009F0AFCC2F
:107E9000552009F0ACCC662009F0A9CC772009F078
:107EA000A6CC882009F0A3CC992009F0A0CC0E9490
:107EB000FD228091A401882309F42FCA2ACB232D07
:107EC0002D3609F07ECE442009F07BCE552009F0F6
:107ED00078CE662009F075CE772009F072CE882022
:107EE00009F06FCE992009F06CCE81E090918B0162
:107EF000911180E080938B01882309F4BDC086E353
:107F000091E000D000D0EF81F885ADB7BEB71296F2
:107F1000FC93EE93119714969C938E9313970E9463
:107F2000FF4E0F900F900F900F908BE891E063E45D
:107F300070E088CE332009F085CA442009F082CA57
:107F4000552009F07FCA662009F07CCA772009F025
:107F500079CA882009F076CA992009F073CA80E0AE
:107F600090E00E94BC0988B192E0892788B9D5C900
:107F7000232D223709F0C6CB442009F0C3CB55206E
:107F800009F0C0CB662009F0BDCB772009F0BACB51
:107F9000882009F0B7CB992009F0B4CB0E940721C3
:107FA000BCC9332009F0BDCD442009F0BACD55201D
:107FB00009F0B7CD662009F0B4CD772009F0B1CD36
:107FC000882009F0AECD992009F0ABCD0E94A629FA
:107FD000A4C9A32DA33609F0C9CD442009F0C6CD0C
:107FE000552009F0C3CD662009F0C0CD772009F0F7
:107FF000BDCD882009F0BACD992009F0B7CD809188
:10800000A501882309F41ECA1092DE0180918A011D
:10801000882309F452CB21E02093D1014ECBA32D2C
:10802000A43609F04DCA442009F04ACA552009F087
:1080300047CA662009F044CA772009F041CA88205F
:1080400009F03ECA992009F03BCA8091A501882316
:1080500009F4F8C931E03093DE012FCB00D0EB8575
:10806000FC85ADB7BEB71296FC93EE9311970E94B4
:10807000FF4E0F900F9021CB89E391E042CF89E32F
:1080800091E0D6CE89E391E0C5CD8091C4018860AE
:108090008093C401C5C880E090E00E94BC0920C95B
:1080A00089B1807408955E9A569A08955E9856989C
:1080B00008955E98569A8DED90E08115910511F026
:1080C0000197F1F72FB7F89456988EE190E081155B
:1080D000910511F00197F1F789B12FBF7894EEEB7C
:1080E000F0E0E115F10511F03197F1F74E9902C07A
:1080F00081E00895807408959FB7F894569AE0E05F
:10810000F0E0E115F10511F03197F1F78111569882
:10811000E5E0F0E0E115F10511F03197F1F74E9B44
:1081200080E0E4E1F0E0E115F10511F03197F1F7BD
:1081300056989FBFEDE0F0E0E115F10511F03197A1
:10814000F1F708950F931F93182F08E0812F817086
:108150000E947C401695811110680150B9F7812F5B
:108160001F910F9108958FEF0E94A2400895DF9212
:10817000EF92FF920F931F93CF93DF93182FEB0192
:108180000E945940882359F0DD24DA948D2DDF9127
:10819000CF911F910F91FF90EF90DF90089580EFA6
:1081A0000E94A240DD2400E498EFE92EE00E0BC00F
:1081B000FF2061F580E00E947C408881869588835D
:1081C00001500E15F9F081E00E947C40F82E81E00C
:1081D0000E947C40882361F7FF2051F4011728F0AA
:1081E000888180FFE7CF101729F3D02EFF24F39466
:1081F0008F2D0E947C4088818695806888830150FD
:108200000E1509F7002311F22196CECF8EEFD82E4E
:10821000BDCF0F931F93CF93DF93182FEB010E94D5
:108220005940209789F085E50E94A24008E0899195
:108230000E94A2400150D9F7812F0E94A240DF91F5
:10824000CF911F910F9108958CEC0E94A240812F35
:108250000E94A240DF91CF911F910F910895DC0100
:10826000CB0181159105A105B10529F08150904000
:10827000A040B040D9F708950F931F93CF93DF9399
:10828000FB01E801608170E0B181A0E06A2B7B2BEB
:10829000803129F177FD34C0DA011C92883289F0EF
:1082A000CB01929582958F7089279F708927F9015C
:1082B00080836F70688380E0DF91CF911F910F9171
:1082C0000895848190E0AC014076507040365105AD
:1082D00039F386FD1CC085FD1CC0687FE1CFDB0142
:1082E000AE7FAA0FBB1FAA0FBB1FAA0FBB1F968191
:1082F0006CE070E0691B71096A0F7B1F77FFCCCFC0
:1083000091E0DA019C93709561957F4FC7CF6E7FA6
:10831000C7CF6C7FC5CF0F931F93CF93DF938C0193
:10832000EB01FC018081BE010E94B740F80180830F
:10833000982F91509D3F28F49881983211F09031F8
:1083400091F7DF91CF911F910F9108951F93CF93D4
:10835000DF93EC010E94594084EBBE010E94094169
:1083600081E00E947C40182F0E94594081E0112337
:1083700009F480E0DF91CF911F9108951F93CF936F
:10838000DF93182FEB010E9459400E945040882330
:1083900029F482E0DF91CF911F91089584E4BE011A
:1083A0000E940941113039F00E94534080E0DF9172
:1083B000CF911F91089580E0DF91CF911F91089593
:1083C0004F925F926F927F928F929F92AF92BF92E5
:1083D000CF92DF92EF92FF920F931F93DF93CF9391
:1083E000CDB7DEB729970FB6F894DEBF0FBECDBF6D
:1083F0005C013B012A0149010E9459408EEBB50105
:108400000E9409418E010F5F1F4F78017AE0C72E4D
:10841000D12CCC0EDD1E0E94B340F70181937F0169
:10842000EC15FD05C1F7C80169E070E00E945943F1
:108430008823C1F083E029960FB6F894DEBF0FBE03
:10844000CDBFCF91DF911F910F91FF90EF90DF9003
:10845000CF90BF90AF909F908F907F906F905F90E4
:108460004F900895F5018081B801A3019201840124
:108470000E943C4180E0DFCF5F926F927F928F92AB
:108480009F92AF92BF92CF92DF92EF92FF920F93A3
:108490001F93DF93CF93CDB7DEB729970FB6F8942C
:1084A000DEBF0FBECDBF582E4B013A0159018EEBF6
:1084B00060E070E00E9409418E010F5F1F4F78015C
:1084C000EAE0CE2ED12CCC0EDD1E0E94B340F70187
:1084D00081937F01EC15FD05C1F7C80169E070E0EB
:1084E0000E9459438823B9F083E029960FB6F89487
:1084F000DEBF0FBECDBFCF91DF911F910F91FF90D7
:10850000EF90DF90CF90BF90AF909F908F907F9033
:108510006F905F900895852DB801A40193018501A6
:108520000E943C4180E0E1CFEF92FF920F931F93B6
:10853000DF93CF93CDB7DEB728970FB6F894DEBFA1
:108540000FBECDBF182F062F7E010894E11CF11C31
:10855000C701A4EBB1E038E00D90FC010192CF011E
:108560003150D1F7242F332727FD309541E752E0D2
:10857000249FC001259F900D349F900D112464E627
:1085800070E00E94AC4BAB0164E6069FB001112481
:10859000460F571FF701CE010996619170E026172B
:1085A0003707B1F0E817F907C1F7112319F0509513
:1085B00041955F4FCA0128960FB6F894DEBF0FBEF3
:1085C000CDBFCF91DF911F910F91FF90EF90089554
:1085D0004F5F5F4FEACF0F931F93DF93CF93CDB7DA
:1085E000DEB72B970FB6F894DEBF0FBECDBF182FA6
:1085F000092F885F612F792F0E94BE41882371F077
:1086000064E371E2CB012B960FB6F894DEBF0FBE88
:10861000CDBFCF91DF911F910F9108956AE673E866
:1086200083E090E00E942F41812F902FBE016F5F69
:108630007F4FAE014E5F5F4F9E012D5F3F4F0E9407
:10864000E0418823E9F69E012C5F3F4FD901ECEA17
:10865000F1E088E001900D928150E1F74B81E42F29
:10866000F0E061E772E0E69FC001E79F900DF69FA2
:10867000900D112464E670E00E94AC4B9A8184E670
:10868000989FC0011124680F791FF901CE010C9643
:108690002191421759F0E817F907D1F7898188230A
:1086A00009F4B0CF709561957F4FACCF6F5F7F4F6E
:1086B000F5CF61157105E1F0E82FF92F20E030E0EA
:1086C00080E0A8E1419198E004C08695915051F076
:1086D0004695542F582750FFF8CF8A2786958068F3
:1086E0009150B1F72F5F3F4F6217730759F7089505
:1086F00080E008951F920F920FB60F920BB60F9263
:1087000011248F93EF93FF938091C600E09125038E
:10871000F0E0EF73F070EA5DFC4F808380912503F9
:108720008F5F80932503FF91EF918F910F900BBE88
:108730000F900FBE0F901F9018951F920F920FB6BB
:108740000F920BB60F9211248F939F93EF93FF9389
:1087500090916603809168039817D1F0E0916803C7
:10876000F0E0EF73F070E759FC4F80818093C60012
:10877000809168038F5F80936803FF91EF919F91D1
:108780008F910F900BBE0F900FBE0F901F901895FA
:108790008091C1008F7D8093C100EFCF1616170620
:1087A0001CF5DC0120E030E0909125038091670307
:1087B0009817D1F3E0916703F0E0EF73F070EA5D92
:1087C000FC4F4081809167038F5F809367034D93D7
:1087D000CD014D3029F02F5F3F4F2617370724F387
:1087E000FC011082C901089520E030E0F9CF8091AA
:1087F000660390916803891B089540E450E09091CE
:10880000660320916803921B9A01291B31092330CA
:108810003105ACF3E0916603F0E0EF73F070E759D7
:10882000FC4F8083809166038F5F80936603809105
:10883000C10080628093C1000895CF93DF93EC0163
:10884000FC018491882341F021960E94FD43FE01A2
:10885000219684918823C9F7DF91CF910895CF9312
:10886000DF93EC018881882331F021960E94FD433B
:1088700089918823D9F7DF91CF9108951F93182FFD
:108880008A3039F0812F0E94FD4380E090E01F91F3
:1088900008958DE00E94FD43812F0E94FD4380E0FA
:1088A00090E01F9108958091250390916703891BA3
:1088B000089590912503809167039817D1F3E09173
:1088C0006703F0E0EF73F070EA5DFC4F80819091F8
:1088D00067039F5F909367030895909125038091AC
:1088E00067039817D1F3E0916703F0E0EF73F0703E
:1088F000EA5DFC4F8081909167039F5F90936703CF
:1089000090E008950E94FD43089585E090E09093E3
:10891000C5008093C40082E08093C0008AE9809300
:10892000C10008958091A9038F5F8093A9038C33C0
:1089300009F008951092A9038091AA038F5F809394
:10894000AA038C33B1F71092AA038091AB038F5F17
:108950008093AB03883169F71092AB038091AC032D
:108960008F5F8093AC038032B9F08F31F1F08E319C
:1089700069F18D31B1F18091AD038D30D1F681E097
:108980008093AD038091AE039091AF0301969093D5
:10899000AF038093AE0308958091AD038F5F809302
:1089A000AD0391E09093AC03E8CF8091AD038430A8
:1089B00031F0863021F0893011F08B30F1F68F5F85
:1089C0008093AD0391E09093AC03D7CF8091AD033A
:1089D000823099F683E08093AD0381E08093AC030D
:1089E00008958091AD03823041F64091AE03E0914D
:1089F000AF03842F9E2F64E670E00E94984B00978F
:108A000051F4842F9E2F60E971E00E94984B8823D7
:108A100009F48FCFDFCF842F8370F9CF0F93DF93CB
:108A2000CF93CDB7DEB760970FB6F894DEBF0FBE19
:108A3000CDBF002309F459C029833A834B835C835B
:108A40006D837E838F839887E0E2E01B29813A81E2
:108A50004B815C811E16BCF019861A861B861C860B
:108A60008E2F992787FD9095909581959F4F04C0F3
:108A7000220F331F441F551F8A95D2F72D873E873B
:108A80004F87588B2AC0CA01B901002E04C0660F57
:108A9000771F881F991F0A94D2F769877A878B8777
:108AA0009C87DA01C90104C0B695A795979587956B
:108AB000EA95D2F72D813E814F81588504C0220F5F
:108AC000331F441F551F0A95D2F7822B932BA42BDB
:108AD000B52B8D879E87AF87B88B29853A854B85C7
:108AE0005C856D857E858F85988960960FB6F89434
:108AF000DEBF0FBECDBFCF91DF910F910895A0E1F2
:108B0000B0E0E5E8F5E40C94E94B29833A834B8324
:108B10005C836D837E838F839887A986BA86CB8694
:108B2000DC86ED86FE860F87188B2D813E814F8176
:108B300058858D859E85AF85B889281739074A07DE
:108B40005B07C8F082179307A407B50790F0298147
:108B50003A814B815C8189859A85AB85BC852817D4
:108B600039074A075B0738F082179307A407B50750
:108B700020F482E003C080E001C081E06096EAE07A
:108B80000C94054C2F923F924F925F926F927F927E
:108B90008F929F92AF92BF92CF92DF92EF92FF920D
:108BA0000F931F93DF93CF93CDB7DEB763970FB6C5
:108BB000F894DEBF0FBECDBF6C017F876E87FC01CE
:108BC00017821682838181FD04C06FC34C855D8549
:108BD00004C01E010894211C311CF6019381EE850E
:108BE000FF8593FD859193FF8191FF87EE87882311
:108BF00009F457C3853241F493FD859193FF819128
:108C0000FF87EE87853259F490E0B6014A8B5B8B83
:108C10000E94D34E4A895B895D874C87D7CF10E08D
:108C2000FF2400E00032B0F48B3269F08C3228F47B
:108C3000803251F0833271F40BC08D3239F08033C1
:108C400049F401602CC00260046029C0086027C09C
:108C5000006125C007FD2EC0282F20532A3098F42C
:108C600006FF08C0812F880F182F110F110F180F42
:108C7000120F15C08F2D880FF82EFF0CFF0CF80E69
:108C8000F20E00620CC08E3221F406FD0AC30064AD
:108C900006C08C3611F4006802C0883659F4EE859F
:108CA000FF8593FD859193FF8191FF87EE87882350
:108CB00009F0B8CF982F9554933018F40061805E76
:108CC00006C0982F9556933008F09BC10F7E06FF83
:108CD00016E06FE3E62EE022853619F4F0E4EF2A81
:108CE00007C0863619F420E8E22A02C0111111509B
:108CF000E7FE06C01C3340F4912E939427E00BC08E
:108D0000183030F4212F06C027E03CE3932E03C037
:108D100027E017E09924CA0104969D878C87FA0101
:108D20006081718182819381A101092D0E94484D4A
:108D30005C016980262D30E0398B288B60FE03C0F2
:108D4000388933FF06C0E1FC06C0E2FE06C000E23F
:108D500005C00DE203C00BE201C000E088899989DB
:108D60008C7090700097C1F1002311F084E001C075
:108D700083E08F1558F4F81AE3FC09C080E290E014
:108D8000B6010E94D34EFA94C9F701C0FF24002314
:108D900029F0802F90E0B6010E94D34E888983FD90
:108DA00003C001ED11E10EC00DEC11E10BC0A114E7
:108DB000B10409F0805290E0B6010E94D34E0F5FDB
:108DC0001F4F05C0AE2CBB2490E1A922BB24F801A3
:108DD0008491882361F762C2E7FE0EC09A0CF8897D
:108DE000F4FF04C08A81813309F49A94191454F56C
:108DF000292D293050F52DC0E6FC2BC0812F90E0A5
:108E00008A159B054CF03CEFA3163FEFB30624F008
:108E100080E8E82A01C01150112349F0E2E0F0E0B7
:108E2000EC0FFD1FE10FF11D80818033A1F3E7FE00
:108E300010C0912E9394812F90E0A816B90644F4A7
:108E40001A1907C09924939404C098E0992E01C080
:108E500010E0E7FE07C01A141B043CF495012F5FD5
:108E60003F4F05C025E030E002C021E030E00023A4
:108E700011F02F5F3F4F112329F0812F90E00196D1
:108E8000280F391F8F2D90E02817390714F4F21A94
:108E900001C0FF244E2C5524C201897090700097A8
:108EA00049F406C080E290E0B6010E94D34EFA94E5
:108EB000FF20C1F7002329F0802F90E0B6010E9427
:108EC000D34E43FC09C006C080E390E0B6010E9487
:108ED000D34EFA94FF20C1F7E7FE46C03501B7FE36
:108EE00002C06624772425010894411C511C4618B1
:108EF0005708420C531CF501E919F1094F01812F64
:108F000090E000271127081B190BFFEF6F16FFEFEA
:108F10007F0629F48EE290E0B6010E94D34EA6149B
:108F2000B70434F0861497041CF4F201808101C068
:108F300080E30894610871080894411C511C601674
:108F400071062CF090E0B6010E94D34EDECF6A1479
:108F50007B0441F49A81963320F4953319F4F8890F
:108F6000F4FF81E390E049C08A81813311F02FEE54
:108F7000622290E0B6010E94D34E112389F08EE266
:108F800090E0B6010E94D34E02E0F101E00FF11D26
:108F90000F5F808190E0B6010E94D34E1150A9F777
:108FA00044FE03C085E490E002C085E690E0B6018F
:108FB0000E94D34EB7FC05C0A114B10441F464FE75
:108FC00006C0B094A194B108B3948DE201C08BE2C5
:108FD00090E0B6010E94D34E80E305C08F5FE6EFBC
:108FE000FFEFAE0EBF1EFAE0AF16B104BCF790E083
:108FF000B6010E94D34EC501C096B6010E94D34E61
:109000004DC1833631F0833789F0833509F059C07B
:1090100022C09A012E5F3F4F3D872C87FA01808145
:109020008983310181E0A82EB12C13C09A012E5FF3
:109030003F4F3D872C87FA016080718006FF03C097
:10904000612F70E002C06FEF7FEFC3010E94334ECB
:109050005C010F7714C09A012E5F3F4F3D872C872C
:10906000FA016080718006FF03C0612F70E002C0CA
:109070006FEF7FEFC3010E94284E5C01006803FD83
:109080001CC006C080E290E0B6010E94D34EFA9464
:109090008F2D90E0A816B906A8F30FC0F30107FDC5
:1090A000859107FF81913F0190E0B6010E94D34E68
:1090B000F110FA940894A108B108A114B10471F751
:1090C000EDC0843611F0893661F507FF0BC09A01B7
:1090D0002C5F3F4F3D872C87FA016081718182812F
:1090E00093810CC09A012E5F3F4F3D872C87FA0178
:1090F00060817181882777FD8095982F0F7697FF83
:1091000008C090958095709561957F4F8F4F9F4FC8
:109110000068A1012AE030E00E94564F982E921874
:1091200041C0853721F40F7E2AE030E020C0097F5E
:109130008F36A9F0803720F4883509F0B2C00BC013
:10914000803721F0883709F0ACC001C0006104FF0E
:1091500009C0046007C004FF08C0066006C028E01C
:1091600030E005C020E130E002C020E132E007FF3E
:109170000AC0CA0104969D878C87FA0160817181BB
:109180008281938109C0CA0102969D878C87FA016A
:109190006081718180E090E0A1010E94564F982E7D
:1091A00092180F7706FF09C00E7F911630F404FF66
:1091B00006C002FD04C00F7E02C0E92C01C0E12EF2
:1091C000802F90E004FF0CC0FE01E90DF11D20810D
:1091D000203311F4097E09C0E39402FF06C004C0E5
:1091E00086789070009709F0E394A02EBB2403FDCD
:1091F00014C000FF0FC0EF1428F4192D1F0D1E1905
:10920000EF2C08C0192D06C080E290E0B6010E9444
:10921000D34EE394EF14C0F304C0EF1410F4FE181F
:1092200001C0FF24A4FE0FC080E390E0B6010E94BD
:10923000D34EA2FE1FC0A1FE03C088E590E010C07F
:1092400088E790E00DC0C50186789070009791F096
:10925000A1FC02C080E201C08BE207FD8DE290E03C
:10926000B6010E94D34E06C080E390E0B6010E9492
:10927000D34E11509116C0F39A94F101E90DF11DEE
:10928000808190E0B6010E94D34E9920A9F706C0D4
:1092900080E290E0B6010E94D34EFA94FF20C1F71D
:1092A00095CCF6012681378102C02FEF3FEFC9012F
:1092B00063960FB6F894DEBF0FBECDBFCF91DF919E
:1092C0001F910F91FF90EF90DF90CF90BF90AF90E4
:1092D0009F908F907F906F905F904F903F902F90D6
:1092E00008955058BB27AA270ED075C166D130F01B
:1092F0006BD120F031F49F3F11F41EF45BC10EF4EA
:10930000E095E7FB51C1E92F77D180F3BA176207E7
:1093100073078407950718F071F49EF58FC10EF45A
:10932000E0950B2EBA2FA02D0B01B90190010C0175
:10933000CA01A0011124FF27591B99F0593F50F48D
:10934000503E68F11A16F040A22F232F342F4427E5
:10935000585FF3CF469537952795A795F0405395DD
:10936000C9F77EF41F16BA0B620B730B840BBAF0AD
:109370009150A1F0FF0FBB1F661F771F881FC2F718
:109380000EC0BA0F621F731F841F48F4879577952C
:109390006795B795F7959E3F08F0B3CF9395880FE3
:1093A00008F09927EE0F979587950895D9D008F47E
:1093B00081E008950CD00FC107D140F0FED030F00D
:1093C00021F45F3F19F0F0C0511139C1F3C014D13D
:1093D00098F39923C9F35523B1F3951B550BBB277C
:1093E000AA2762177307840738F09F5F5F4F220F29
:1093F000331F441FAA1FA9F333D00E2E3AF0E0E822
:1094000030D091505040E695001CCAF729D0FE2F6D
:1094100027D0660F771F881FBB1F261737074807FF
:10942000AB07B0E809F0BB0B802DBF01FF279358B5
:109430005F4F2AF09E3F510568F0B6C000C15F3F04
:10944000ECF3983EDCF3869577956795B795F7959D
:109450009F5FC9F7880F911D9695879597F9089595
:10946000E1E0660F771F881FBB1F62177307840731
:10947000BA0720F0621B730B840BBA0BEE1F88F740
:10948000E095089504D06894B111D9C00895BCD076
:1094900088F09F5790F0B92F9927B751A0F0D1F0DD
:1094A000660F771F881F991F1AF0BA95C9F712C067
:1094B000B13081F0C3D0B1E00895C0C0672F782FDC
:1094C0008827B85F39F0B93FCCF3869577956795D3
:1094D000B395D9F73EF490958095709561957F4F3F
:1094E0008F4F9F4F0895E89409C097FB3EF49095E5
:1094F0008095709561957F4F8F4F9F4F9923A9F06D
:10950000F92F96E9BB279395F695879577956795FB
:10951000B795F111F8CFFAF4BB0F11F460FF1BC03F
:109520006F5F7F4F8F4F9F4F16C0882311F096E9D2
:1095300011C0772321F09EE8872F762F05C0662380
:1095400071F096E8862F70E060E02AF09A95660F39
:10955000771F881FDAF7880F9695879597F90895F2
:10956000990F0008550FAA0BE0E8FEEF1616170634
:10957000E807F907C0F012161306E407F50798F09C
:10958000621B730B840B950B39F40A2661F0232BB5
:10959000242B252B21F408950A2609F4A140A69531
:1095A0008FEF811D811D089597F99F6780E870E016
:1095B00060E008959FEF80EC089500240A94161649
:1095C000170618060906089500240A9412161306B1
:1095D000140605060895092E0394000C11F488233F
:1095E00052F0BB0F40F4BF2B11F460FF04C06F5F5B
:1095F0007F4F8F4F9F4F089557FD9058440F551F31
:1096000059F05F3F71F04795880F97FB991F61F004
:109610009F3F79F087950895121613061406551F7B
:10962000F2CF4695F1DF08C0161617061806991FE7
:10963000F1CF86957105610508940895E894BB27DC
:1096400066277727CB0197F908958ADF08F48FEF13
:1096500008950BD0C0CFB1DF28F0B6DF18F0952306
:1096600009F0A2CFA7CF1124EACFC6DFA0F3959FC0
:10967000D1F3950F50E0551F629FF001729FBB27F9
:10968000F00DB11D639FAA27F00DB11DAA1F649FA5
:109690006627B00DA11D661F829F2227B00DA11D58
:1096A000621F739FB00DA11D621F839FA00D611DDE
:1096B000221F749F3327A00D611D231F849F600DFF
:1096C000211D822F762F6A2F11249F5750408AF038
:1096D000E1F088234AF0EE0FFF1FBB1F661F771FC4
:1096E000881F91505040A9F79E3F510570F05CCF04
:1096F000A6CF5F3FECF3983EDCF3869577956795B0
:10970000B795F795E7959F5FC1F7FE2B880F911DE1
:109710009695879597F90895991B79E004C0991F4C
:10972000961708F0961B881F7A95C9F780950895BB
:10973000AA1BBB1B51E107C0AA1FBB1FA617B70777
:1097400010F0A61BB70B881F991F5A95A9F7809593
:109750009095BC01CD01089597FB092E07260AD0EC
:1097600077FD04D0E5DF06D000201AF470956195EE
:109770007F4F0895F6F7909581959F4F0895A1E248
:109780001A2EAA1BBB1BFD010DC0AA1FBB1FEE1F7B
:10979000FF1FA217B307E407F50720F0A21BB30BC6
:1097A000E40BF50B661F771F881F991F1A9469F742
:1097B00060957095809590959B01AC01BD01CF019E
:1097C00008952F923F924F925F926F927F928F9265
:1097D0009F92AF92BF92CF92DF92EF92FF920F9340
:1097E0001F93CF93DF93CDB7DEB7CA1BDB0B0FB64A
:1097F000F894DEBF0FBECDBF09942A883988488807
:109800005F846E847D848C849B84AA84B984C8849C
:10981000DF80EE80FD800C811B81AA81B981CE0F93
:10982000D11D0FB6F894DEBF0FBECDBFED01089578
:109830002F923F924F925F926F927F929F92AF9240
:10984000BF92CF92DF92EF92FF920F931F93CF932D
:10985000DF933B01EA016115710519F0FB0180837B
:109860009183209739F09E012250304023323105F8
:1098700008F0D5C0C82ED92EF60111916F017F01D5
:10988000812F90E00E94204E0097B1F71D3231F4F5
:10989000F60111917F019924939406C01B3219F4AB
:1098A000F60111917F019924209719F0C031D1055B
:1098B000D1F4103389F4F7018081883711F08835AD
:1098C00059F4F701118182E090E0E80EF91E92E070
:1098D000992AC0E1D0E007C0209729F41033B1F0F5
:1098E000CAE0D0E02BC0CA30D10541F1C031D1056A
:1098F00021F0C830D105A9F409C02FEFA22E2FEF17
:10990000B22E2FEFC22E2FE0D22E20C0C8E0D0E022
:109910009FEFA92E9FEFB92E9FEFC92E9FE1D92E61
:1099200015C09E01442737FD4095542F6FEF7FEF00
:10993000CB010E94BF4B59016A0108C089E9A82EDA
:1099400089E9B82E89E9C82E89E1D82E60E020E0A7
:1099500030E0A9011E01442437FC4094542C012F0F
:1099600000530A3060F0812F81548A3110F407507F
:1099700006C0812F81568A3150F5012F0755802F5F
:1099800090E08C179D071CF56F3FE9F0A216B30617
:10999000C406D506A8F0CA01B901A20191010E942E
:1099A000E4529B01AC01802F90E0A0E0B0E0280FD2
:1099B000391F4A1F5B1F281739074A075B0710F436
:1099C0006FEF01C061E0F70111917F01C8CF611411
:1099D000710481F0662339F00894E108F108F3017D
:1099E000F182E08207C091FE05C0C7010297F30132
:1099F0009183808390FE07C05095409530952195C6
:109A00003F4F4F4F5F4F67FF0DC082E290E0909352
:109A1000B7038093B6032FEF3FEFA90103C020E007
:109A200030E0A901B901CA01DF91CF911F910F91D7
:109A3000FF90EF90DF90CF90BF90AF909F907F907E
:109A40006F905F904F903F902F90089566277727F3
:109A50000C943451FC0188279927E89421912032F5
:109A6000E9F3293010F02E30C8F32B3241F02D32BB
:109A700039F4689404C00E943E4E820F911D2191DA
:109A800020532A30C0F31EF4909581959F4F08957E
:109A9000283008F027E03327DA01990F311D87FDC0
:109AA000916000966105710539F432602E5F3D9337
:109AB00030E32A95E1F708959F3F30F08038710533
:109AC000610509F03C5F3C5F3D93913008F0806890
:109AD000911DDF93CF931F930F93FF92EF92192F56
:109AE000987F9695E92F96959695E90FFF27E15D6A
:109AF000FD4E99273327EE24FF24A701E7010590A7
:109B00000894079428F4360FE71EF81E491F511DCC
:109B1000660F771F881F991F0694A1F70590079479
:109B200028F4E70EF81E491F561FC11D770F881F26
:109B3000991F661F0694A1F70590079428F4F80E64
:109B4000491F561FC71FD11D880F991F661F771FFA
:109B50000694A1F70590079420F4490F561FC71FDC
:109B6000D81F990F661F771F881F0694A9F7849145
:109B70001095177041F0D695C79557954795F7946E
:109B8000E7941A95C1F7E5EDF1E168941590159108
:109B900035916591959105907FE27395E118F10AF1
:109BA000430B560BC90BD009C0F7E10CF11E431F44
:109BB000561FC91FD01D7EF4703311F48A95E6CF6D
:109BC000E894015030F0080F0AF40027021708F457
:109BD000202F2395022F7A3328F079E37D932A955D
:109BE000E9F710C07D932A9589F6069497956795B5
:109BF000379517951794E118F10A430B560BC90BCB
:109C0000D00998F023957E9173957A3308F070E32C
:109C10007C932013B8F77E9170617D9330F083952B
:109C200071E37D9370E32A95E1F71124EF90FF90A3
:109C30000F911F91CF91DF91992787FD90950895FE
:109C40009111A0C4803219F089508550D0F7089541
:109C5000FC010590615070400110D8F780959095F7
:109C60008E0F9F1F0895FC016150704001900110FC
:109C7000D8F7809590958E0F9F1F08957AE0979F53
:109C8000902D879F802D910D112408950F931F9380
:109C9000CF93DF938C01EB01009711F42097C9F16A
:109CA00081E090E06EE070E00E94DC4FFC019C01DE
:109CB000009789F180E88383209771F0D387C2876A
:109CC00081E883838091B0039091B103009721F4E0
:109CD000F093B103E093B00301151105E1F0118792
:109CE00000878381826083838091B2039091B30364
:109CF000009789F4F093B303E093B2038091B40327
:109D00009091B503009739F4F093B503E093B40351
:109D100002C020E030E0C901DF91CF911F910F9187
:109D20000895CF93DF93EC013B8130FF36C036FFBF
:109D300009C03F7B3B838E819F8101969F838E83E9
:109D40002A8129C032FF0FC0E881F98180819927DB
:109D500087FD9095009719F430623B831EC03196C1
:109D6000F983E88311C0EA85FB85CE01099597FF49
:109D70000BC02B813FEF8F3F930711F480E101C0AF
:109D800080E2822B8B8309C02E813F812F5F3F4F62
:109D90003F832E83282F30E002C02FEF3FEFC90111
:109DA000DF91CF9108950F931F93CF93DF938C0191
:109DB000EB018B8181FF1BC082FF0DC02E813F8193
:109DC0008C819D812817390764F4E881F98101931A
:109DD000F983E88306C0E885F985802F0995009707
:109DE00031F48E819F8101969F838E8302C00FEF95
:109DF0001FEFC801DF91CF911F910F910895DF935D
:109E0000CF93CDB7DEB7FE01359661917191809108
:109E1000B2039091B303DC0113962C911397286041
:109E200013962C93AF010E94C245E091B203F091CA
:109E3000B3032381277F2383CF91DF910895EF928E
:109E4000FF920F931F93CF93DF938C01E091B203A6
:109E5000F091B303838181FF1FC0C0E0D0E00AC04E
:109E6000DB011896ED91FC9119970995009711F077
:109E7000CFEFDFEFF80181918F016091B203709114
:109E8000B303882369F7DB011896ED91FC911997CC
:109E90008AE00995009711F0CFEFDFEFCE01DF9157
:109EA000CF911F910F91FF90EF900895FA01AA278B
:109EB000283051F1203181F1E8946F936E7F6E5F0D
:109EC0007F4F8F4F9F4FAF4FB1E03ED0B4E03CD0BB
:109ED000670F781F891F9A1FA11D680F791F8A1F9E
:109EE000911DA11D6A0F711D811D911DA11D20D005
:109EF00009F468943F912AE0269F11243019305DBF
:109F00003193DEF6CF010895462F4770405D4193AF
:109F1000B3E00FD0C9F7F6CF462F4F70405D4A33FC
:109F200018F0495D31FD4052419302D0A9F7EACFC4
:109F3000B4E0A6959795879577956795BA95C9F7F3
:109F400000976105710508959B01AC010A2E0694E6
:109F50005795479537952795BA95C9F7620F731F9F
:109F6000841F951FA01D0895DC01CB01FC01F99908
:109F7000FECF06C0F2BDE1BDF89A319600B40D9255
:109F800041505040B8F70895DC01CB0103C02D913A
:109F90000E94CF4F41505040D0F70895262FF99995
:109FA000FECF1FBA92BD81BD20BD0FB6F894FA9ABC
:109FB000F99A0FBE01960895EF92FF920F931F93A7
:109FC000CF93DF93689F8001699F100D789F100DDC
:109FD0001124C8010E940150E82EE7017E01F92EEC
:109FE000E701209731F08E2D60E070E0A8010E941B
:109FF000DD52CE01DF91CF911F910F91FF90EF9035
:10A000000895CF93DF938230910510F482E090E0C1
:10A01000E091BA03F091BB0340E050E020E030E073
:10A0200026C06081718168177907E0F068177907A9
:10A0300081F4828193812115310531F0D901139684
:10A040009C938E9312972BC09093BB038093BA037B
:10A0500026C04115510519F06417750718F4AB01B6
:10A06000E901DF019F0172816381E72FF62F3097AD
:10A07000C1F64115510501F1481B590B44305105FA
:10A0800080F412968D919C911397209719F09B83E1
:10A090008A8304C09093BB038093BA03FD01329678
:10A0A00046C0FD01E40FF51F81939193425050404B
:10A0B00011965C934E933BC02091B8033091B90345
:10A0C0002115310541F42091BE013091BF0130933B
:10A0D000B9032093B8032091C0013091C10121152B
:10A0E000310541F42DB73EB74091BC015091BD01FF
:10A0F000241B350BE091B803F091B903E217F30785
:10A10000A0F42E1B3F0B2817390778F0AC014E5FE7
:10A110005F4F2417350748F04E0F5F1F5093B90368
:10A120004093B8038193919302C0E0E0F0E0CF0147
:10A13000DF91CF910895CF93DF93009709F491C0F9
:10A14000FC013297138212826091BA037091BB03B3
:10A150006115710581F420813181280F391F8091AB
:10A16000B8039091B9038217930799F5F093B90357
:10A17000E093B80376C0DB0180E090E002C0CD013F
:10A18000D901AE17BF0748F412962D913C91139751
:10A1900021153105A1F7CD0121C0B383A283EF01C1
:10A1A000499159919E01240F351FA217B30779F4E5
:10A1B0002D913C911197240F351F2E5F3F4F318316
:10A1C000208312962D913C9113973383228300971D
:10A1D00029F4F093BB03E093BA0343C0DC01139668
:10A1E000FC93EE9312974D915D91A40FB51FEA1762
:10A1F000FB0769F420813181240F351F2E5F3F4F0B
:10A20000EC0139832883228133813B832A83E0E078
:10A21000F0E002C0FB01BC01DB0112968D919C9124
:10A2200013970097B9F79B012E5F3F4F8D919C913B
:10A230001197820F931F4091B8035091B9034817AB
:10A24000590779F4309729F41092BB031092BA039E
:10A2500002C013821282225030403093B9032093FF
:10A26000B803DF91CF9108956F927F928F929F9262
:10A27000AF92BF92CF92DF92EF92FF920F931F9314
:10A28000DF93CF930F92CDB7DEB75B0161157105F8
:10A2900021F0DB018C9311969C93482F592F6A0172
:10A2A000F601E1906F018F018E2D90E00E94204E0B
:10A2B0000097B1F7FE2DFD3229F4D601ED908D0106
:10A2C00021E007C0BE2DBB3219F4F601E1908F01E9
:10A2D00020E068010894C108D108C6016FEC72E162
:10A2E00043E050E029830E94C5522981009711F56F
:10A2F00072E0E72EF12CE00EF11EC70162ED72E173
:10A3000045E050E00E94C5522981009729F467E09A
:10A31000E62EF12CE00EF11EA114B10421F0D501BE
:10A320001196FC92EE9220FF0FC130E020E090E801
:10A330008FEF12C1C60167ED72E143E050E029835F
:10A340000E94C5522981009731F060E070E0CB0196
:10A35000662477240AC0A114B10409F4F9C00E5F81
:10A360001F4FF50111830083F3C03E2D30533A3067
:10A37000A0F52260E22FF0E0AF014870507022FF9C
:10A3800007C04115510571F50894611C711C2AC064
:10A390004115510519F00894610871086B017C01A1
:10A3A00052E0CC0CDD1CEE1CFF1C5A95D1F76C0D55
:10A3B0007D1D8E1D9F1D660F771F881F991F630FC0
:10A3C000711D811D911D6839F9E97F07F9E98F0732
:10A3D000F9E19F0738F0246005C03E3F39F423FDC2
:10A3E0003FC02860D801ED908D01BFCF353311F00B
:10A3F0003531B1F5F80131913D3211F4206102C0DF
:10A400003B3241F4D80111963C911197319642E0CC
:10A4100050E002C041E050E030533A3020F08F016C
:10A42000041B150B1DC040E050E0BCE040385B074A
:10A430005CF4DA01AA0FBB1FAA0FBB1F4A0F5B1FF8
:10A44000440F551F430F511D319130538F013A3046
:10A4500060F324FF03C0509541955F4F640E751E55
:10A46000C22EDD2421FF08C0A114B10429F001503F
:10A470001040F501118300830E94734A7B018C0117
:10A48000F3E0CF22DD2433E0C316D10421F417FB1F
:10A49000109517F91095C801B70120E030E0A90127
:10A4A0000E94D649882309F44AC077FE09C04EEEBF
:10A4B000C42E42E1D42E709461947108739404C048
:10A4C00036E0C32E33E1D32E26E0822E912C90E28B
:10A4D000A92EB12C0FC0F6012591359145915491CB
:10A4E000C801B7010E94294BE62EF72E082F192F1D
:10A4F0006A187B086A147B0474F7B594A7940894CF
:10A50000810891088114910429F08CEF9FEFC80E07
:10A51000D91EF0CFB701C801282F220F292F221FE3
:10A520002F3F39F020E030E0A9010E94D64988236E
:10A5300031F482E290E09093B7038093B6033E2D0E
:10A540002F2D902F812F08C030E020E090E803C02D
:10A5500030E020E090EC8FE7F901AC016F2F722F13
:10A56000852F942F0F90CF91DF911F910F91FF9026
:10A57000EF90DF90CF90BF90AF909F908F907F90A3
:10A580006F900895992788270895FB01DC014150B9
:10A59000504088F08D9181341CF08B350CF4805E36
:10A5A000659161341CF06B350CF4605E861B6111A3
:10A5B00071F3990B0895881BFCCFDC0101C06D93EA
:10A5C00041505040E0F70895629FD001739FF00121
:10A5D000829FE00DF11D649FE00DF11D929FF00D33
:10A5E000839FF00D749FF00D659FF00D9927729F6A
:10A5F000B00DE11DF91F639FB00DE11DF91FBD01F5
:0AA60000CF0111240895F894FFCF54
:10A60A0028457874507772290000617478707772DF
:10A61A006F6B005874616C00496E7465726E0057F6
:10A62A0061746368646F67004E6F726D616C004F8E
:10A63A004E004F4646004F6E004F666600486967F7
:10A64A0068004C6F770001010000C841AE47E13C49
:10A65A00AE47E13CAE47E13C0AD7A33B0AD7A33B4E
:10A66A000533332341000090410000584166666675
:10A67A00410000A0400000204100004041CDCC4CE8
:10A68A003F0A00007A455802050001010000FF0355
:10A69A008A000400000000000000FF038800050093
:10A6AA00000000001A010114030500010203060755
:10A6BA000A0B0E0F020306070A0B0E0F2000BD033A
:02A6CA0000008E
:00000001FF
